:100000000C94BB010C94CD010C94CD010C94C22E28
:100010000C94B22B0C94CD010C94CD010C94CD0119
:100020000C94CD010C94CD010C94CD010C9487322D
:100030000C94CD010C94CD010C94CD010C94CD0108
:100040000C943B320C94CD010C9483030C9413025A
:100050000C94CD010C94CD010C94CD010C94CD01E8
:100060000C94CD010C94CD01B903BB03F403F4034C
:10007000F403F403F403F403F403F403F403F403C8
:10008000C103C303C503C703C903CB03CD03CF0318
:10009000F403D303D503D703D903DB03DD03F40350
:1000A000DF03C908CF08D208D508DA08E208EA0851
:1000B000850985098509F708FA0803090C098509E6
:1000C00085098509850985098509180922092E09E7
:1000D0003609390942094B095109850985095A0927
:1000E00063096E099F0B32173217A90BB40BBF0BB4
:1000F000CA0B3217CE0B3217DC0B3217E60BF00BA4
:10010000FA0B3217321732170A0C170C240C084A54
:10011000D73B3BCE016E84BCBFFDC12F3D6C74311B
:100120009ABD56833DDA3D00C77F11BED9E4BB4C72
:100130003E916BAAAABE000000803F05A84CCDB23C
:10014000D44EB93836A9020C50B9918688083CA61D
:10015000AAAA2ABE000000803F000D0A4772626C06
:1001600020312E3167205B27242720666F7220689C
:10017000656C705D0D0A00244E005B4F50543A00D0
:100180005B5645523A312E31672E3230313831319B
:1001900031323A005B544C4F3A005B4739323A00F7
:1001A0003330003238005B4700204700204D0020EC
:1001B000530020460020540033382E005B47433A5A
:1001C00047005B484C503A24242024232024472015
:1001D000244920244E2024783D76616C20244E78DA
:1001E0003D6C696E6520244A3D6C696E6520245320
:1001F0004C50202443202458202448207E202120B5
:100200003F206374726C2D785D0D0A00536C656538
:1002100070696E6700526573746F72696E672073E0
:1002200070696E646C6500526573746F72696E6795
:100230002064656661756C74730050676D20456E4F
:100240006400436865636B204C696D697473004397
:100250006865636B20446F6F720044697361626C00
:10026000656400456E61626C656400436175746924
:100270006F6E3A20556E6C6F636B6564002724487F
:10028000277C2724582720746F20756E6C6F636B52
:1002900000526573657420746F20636F6E74696EAD
:1002A0007565005B4D53473A00414C41524D3A0051
:1002B0007C413A007C4F763A007C57434F3A007CB1
:1002C000506E3A007C46533A007C42663A007C57B6
:1002D000506F733A007C4D506F733A00536C6565F4
:1002E0007000446F6F723A00436865636B00416C45
:1002F00061726D00486F6D65004A6F6700486F6CF2
:10030000643A0052756E0049646C650000007A43DF
:1003100000007A4300007A430000FA430000FA43E9
:100320000000FA4300A00C4700A00C4700A00C47B7
:10033000000048C3000048C3000048C30A0000FF93
:10034000010AD7233C6F12033B00007A44000000EF
:100350000004000000C8410000FA43FA00000080D9
:100360003F0D0A005B5052423A006572726F723A5A
:10037000006F6B0D0A0011241FBECFEFD8E0DEBF67
:10038000CDBF27E0A0E0B1E001C01D92A136B207C9
:10039000E1F70E9468040C946B3A0C940000CF9330
:1003A000DF93239AC0EBD0E083E0888384E08093DE
:1003B000B100259A20915C0230915D0240915E026D
:1003C00050915F02609158027091590280915A02D7
:1003D00090915B020E949B359B01AC0160E070E054
:1003E0008EE793E40E949B366093000170930101B5
:1003F000809302019093030188818F778883DF9136
:10040000CF9108950E94CA1C0E94B61B80910B02D6
:10041000811108C00E94671D892BB1F780910A02E3
:10042000883091F308951F920F920FB60F92112406
:100430008F939F93EF93FF9380916E01E82FF0E0ED
:10044000EB5FFE4F90819093C6008F5F893609F471
:1004500080E080936E0190910401891305C0809122
:10046000C1008F7D8093C100FF91EF919F918F918B
:100470000F900FBE0F901F901895E091040191E02E
:100480009E0F993631F490E004C020910D0724FDB1
:100490000FC020916E012917C1F3F0E0EB5FFE4F12
:1004A0008083909304018091C10080628093C10099
:1004B000089590910B02911107C086FF02C0439AE4
:1004C00001C043981092150208954F925F926F9267
:1004D0007F928F929F92AF92BF92CF92DF92EF92D4
:1004E000FF926B017C0180905C0290905D02A09075
:1004F0005E02B0905F0240905802509059026090A6
:100500005A0270905B02A3019201C501B4010E94DE
:10051000B33887FF19C06091130270E080E090E06B
:100520000E9445372AE037ED43E25CE30E94F3384E
:10053000A70196010E94F3386B017C01A30192018F
:100540000E94B33887FD0AC04092170250921802E9
:100550006092190270921A028FEF47C0A5019401B0
:10056000C701B6010E9491361816E4F020E030E091
:10057000A901C701B6010E949136811109C01092EC
:100580001702109218021092190210921A022DC02E
:100590008092170290921802A0921902B0921A0249
:1005A00081E023C0C0921702D0921802E092190293
:1005B000F0921A02A5019401C701B6010E949B3571
:1005C00020910001309101014091020150910301FD
:1005D0000E94F3380E94803720E030E040E85FE37B
:1005E0000E949C350E941437862FFF90EF90DF9079
:1005F000CF90BF90AF909F908F907F906F905F90C3
:100600004F9008958093B300811104C08091B00091
:100610008F7703C08091B00080688093B000089508
:1006200090910B02911126C081110EC010921702F9
:10063000109218021092190210921A028091B000C2
:100640008F778093B00014C0803111F42D9801C0D1
:100650002D9A9091600291FF05C0803219F440E01C
:1006600050E0BA01CB01BA010E9465020E94020368
:10067000109215020895CF92DF92EF92FF92CF93DE
:1006800090910A02923079F06A017B01C82F0E9492
:100690000202B701A6018C2FCF91FF90EF90DF905F
:1006A000CF900C941003CF91FF90EF90DF90CF90FC
:1006B000089561EF71E088E892E00C94622B8091DC
:1006C0000D0784FD1FC080E10E941E2B8091B000A9
:1006D0008F778093B000439890910A02892F8C7293
:1006E00021F480910E02867069F0943031F480918B
:1006F0000E07811105C086E001C083E00E940E2B29
:100700000C94513208951F920F920FB60F9211243C
:100710002F933F934F935F936F937F938F939F9309
:10072000AF93BF93EF93FF93E091C600E13271F076
:1007300028F4E83179F40E945F0356C0EF3321F0CA
:10074000EE3741F482E003C081E001C088E00E94FE
:100750001E2B4AC0E7FF37C08E2F90E0FC01E45803
:10076000F109ED31F10508F03FC0EC5CFF4F0C944E
:100770003E3A80E2ECCF80910A0285FF35C080E4EA
:10078000E6CF81E00DC082E00BC084E009C088E0C4
:1007900007C080E105C080E203C080E401C080E8BA
:1007A0000E94052B21C081E00BC082E009C084E0DB
:1007B00007C088E005C080E103C080E201C080E49A
:1007C0000E94FC2A11C0A091EA0281E08A0F8138C0
:1007D00009F480E09091EB02891731F0B0E0A15963
:1007E000BE4FEC938093EA02FF91EF91BF91AF91DE
:1007F0009F918F917F916F915F914F913F912F9139
:100800000F900FBE0F901F901895FF920F931F939C
:10081000CF93DF938C01EB018091600285FF26C0AE
:10082000F0900A0280E2F81629F1C8010E94272BF5
:100830008823E1F081E080930D0288E0F81641F012
:100840000E945F0382E00E940E2B0E94B61B0EC026
:1008500088E00E941E2B0E94B61B80910B02811122
:1008600005C080910A028111F6CFEACF80910A0279
:10087000823041F10E94B61B80910B02811122C08F
:100880009091CA038091C903981303C00E94CA1CA7
:10089000F1CFBE01C8010E94DA27811113C08091F7
:1008A000600281FF0FC0888584FF0CC04C815D8190
:1008B0006E817F8180E1DF91CF911F910F91FF9039
:1008C0000C943B03DF91CF911F910F91FF900895FE
:1008D000CF93DF93CDB7DEB761970FB6F894DEBF45
:1008E0000FBECDBF8091C00082608093C000109287
:1008F000C50080E18093C4008091C1008869809325
:10090000C10080E090E00E94431E8A3009F038C5A3
:1009100045E550E061E070E08BE192E00E944B1E03
:10092000892B09F42DC58AB18C618AB9209A8AB1C4
:10093000806E8AB9809181008F7E80938100809142
:100940008100886080938100809180008C7F8093FB
:100950008000809180008F708093800080916E0075
:10096000887F80936E0014BC15BC80916E008160FE
:1009700080936E0087B1887F87B988B1876088B916
:1009800080916C00876080936C0080916800826029
:10099000809368008CE0E1EFF1E0DF011D928A9521
:1009A000E9F7789410920A028091600284FF03C0F4
:1009B00081E080930A02AAE02A2EA2E03A2E99242E
:1009C000939480910A0291E1F10111929A95E9F7CD
:1009D00080930A0284E6809311028093120280932E
:1009E00013028CE0ADEFB1E01D928A95E9F7109209
:1009F000090210920D0710920E0710920F07109225
:100A000010078091EA028093EB0280E4E0E7F2E0D5
:100A100011928A95E9F764E972E080E00E948F1EE6
:100A2000811103C087E00E940B2D0E94CF013B9AE9
:100A300043980E940C313D98459A80E00E94EC2B2F
:100A40000E94771D0E949A2A0E940F320E94590329
:100A50008AE591E00E94F82C8091600283FF10C02B
:100A60000E94F12E882361F090920A0283EA92E0BC
:100A70000E94F82C82E492E00E94F82C0E94932EAF
:100A800080910A02817899F083EA92E00E94F82C22
:100A90008DE792E00E94F82C0E94932E90920A0219
:100AA00010E000E0E2E0EE2EF4E08F2E29C010927C
:100AB0000A020E941F2DF4CFE92FF0E0E159FE4F0A
:100AC00080819F5F913809F490E09093EB028F3F13
:100AD000E9F08A3021F50E94B61B80910B0281114A
:100AE00070CFE12FF0E0EF5EF84F1082F02FF17041
:100AF000FF2E00FF18C08BE00E940B2D10E000E0DD
:100B00009091EB028091EA029813D6CF0E94CA1C02
:100B10000E94B61B80910B02882391F352CF8D3037
:100B200009F008C4D8CF80911107882309F4FFC3C6
:100B3000843209F0F4C3998A80911207833409F151
:100B400034F4882361F0843209F006C11AC08A3473
:100B500059F08835B1F0873409F0FEC012C082EC3C
:100B600091E00E94F82CD9C380910A028F7D09F090
:100B7000C4C3809113078D3309F0C7C30E94C9090C
:100B8000BFC3909113079111C0C3833409F4B2C05D
:100B90001CF4843239F0C1C3873469F0883509F414
:100BA000C9C0BBC380910A028871F82E09F0A5C3A1
:100BB0000E94812DB2C38CEB91E00E94F82C8091B1
:100BC00070028C3838F088EB91E00E94F82C80910C
:100BD00070028A580E94D22C89EA91E00E94F82C77
:100BE000809176028A5C0E94D22C89EA91E00E9470
:100BF000F82C809174028F5E0E94D22C89EA91E0D9
:100C00000E94F82C8091720225E1281B822F0E94FD
:100C1000D22C89EA91E00E94F82C80917302865AC6
:100C20000E94D22C89EA91E00E94F82C80917102F6
:100C30009EE5981B892F0E94D22C809177028823F1
:100C400099F08CEA91E00E94F82C80917702833031
:100C500029F08E3139F0823039F404C080E30E94EB
:100C60003D0202C00E94D22C8CEA91E00E94F82C36
:100C700080917902803131F0803231F0811107C0EA
:100C800085E303C083E301C084E30E943D028CEA54
:100C900091E00E94F82C80917802882311F088E37B
:100CA00001C089E30E943D0285EB91E00E94F82C8F
:100CB000809183020E94D22C82EB91E00E94F82C5A
:100CC00060917F02709180028091810290918202F6
:100CD0000E949B2C8FEA91E00E94F82C60917B028D
:100CE00070917C0280917D0290917E0240E00E9492
:100CF000FE2B0EC080910A02823069F40E945F03CD
:100D000083EA92E00E94F82C8AE592E00E94F82C97
:100D10000E94932E02C38111F0C2E0920A0283EA7C
:100D200092E00E94F82C83E692E00E94F82C0E9448
:100D3000932E3BC080910A02813009F0EEC283EA13
:100D400092E00E94F82C8BE692E00E94F82C0E9420
:100D5000932E10920A02E1C290910A02923008F09A
:100D6000CCC2893409F49FC034F4833271F08834E2
:100D700009F45AC041C1823509F4E8C0833509F449
:100D800080C08E3409F038C111C1809113078111E0
:100D9000BCC210E0BE016F5F7F4F812F0E948F1E8B
:100DA000811105C087E00E940B2DF12CB6C286EAA6
:100DB00091E00E94F82C163029F0173041F480EAB7
:100DC00091E002C083EA91E00E94F82C04C086E31F
:100DD000810F0E94D22C8AE30E943D02CE0101962F
:100DE0000E94B92C0E94932E1F5F183099F68AE951
:100DF00091E00E94F82C80EA92E00E94B92C0E94B7
:100E0000932E84E991E00E94F82C6091AC027091DD
:100E1000AD028091AE029091AF020E94AA2C0E9476
:100E2000932E0E94982E79C28091600284FF62C244
:100E300080920A0280911307811167C20E940131DA
:100E400084E00E94062F83E00E94062F0E94B61BBA
:100E500080910B02811106C00E9459030E940F323B
:100E60000E940C3180910B02811157C210920A022C
:100E70000E9451328091130781114FC20E941F2D91
:100E800094CF809113078C3409F03FC280911407EE
:100E9000803509F03AC280911507811136C280E889
:100EA0000E941E2B3AC2E98A80911307811130C03B
:100EB00040E550E06EEA73E081E197E00E944B1E4E
:100EC000892B51F41092110740E550E061E177E081
:100ED0008EEA93E00E94881D80E891E00E94F82C41
:100EE0000E94CD2A0E94932E8AE791E00E94F82C5E
:100EF00086E50E943D028CE20E943D028FE00E9446
:100F0000D22C8CE20E943D0280E80E94D22C00CFBD
:100F1000A3E0A98B8D3309F0F8C183E0282F30E0DE
:100F2000F901EF5EF84F9081D901A25FB84F9C9311
:100F30008F5F90819111F2CF898B40E550E061E1A4
:100F400077E08EEA93E00E94881DE7C18091130745
:100F5000833509F0DAC180911407843509F0D5C1D1
:100F6000809115078D3309F0D0C180911707811149
:100F7000CCC180911607843239F08A3239F083323D
:100F800009F0C3C182E003C081E001C08FEF0E947D
:100F9000E61D83EA92E00E94F82C87E292E00E942C
:100FA000F82C0E94932E0E945F03B7C1E98A8091BA
:100FB000130781111DC010E0812F0E94DA2A8111D0
:100FC00004C087E00E940B2D0EC087E791E00E94CD
:100FD000F82C812F0E94D22C8DE30E943D020E94AA
:100FE000CD2A0E94072D1F5F123009F496C1E4CF6D
:100FF000911183C111E001C010E0BE01635F7F4F1A
:10100000CE0141960E94E734811103C072E0F72EB1
:1010100084C1E98981E08E0F898BF0E0EF5EF84FA3
:1010200090819D3309F071C1112371F1482F50E077
:10103000282F30E0F901EF5EF84F9081241B350B2B
:10104000D901AF5EB84F9C938F5F90819111F0CF23
:10105000898B0E94C909811153C16D857E858F8559
:1010600098890E94D6390E941437162F0E940202D6
:10107000B1E51B9FC001112440E550E061E177E03C
:101080009D5F0E94881D91CEBE016F5F7F4FCE0194
:1010900041960E94E734882309F4B8CFE989F0E04B
:1010A000EF5EF84F8081811130C1AD84BE84CF8462
:1010B000D88820E030E04FE753E4C601B5010E9434
:1010C000B33818160CF421C149805A806B807C809B
:1010D000C601B5010E941437062F20E030E0A901B7
:1010E000C301B2010E94913687FD0CC1043608F499
:1010F00040C0045680E0033098F510E0000F111F47
:10110000000F111F823079F0F801833011F1813026
:1011100019F0E55EFD4F02C0E95DFD4F408251824E
:1011200062827382E4C00D5C1D4F20E030E040E736
:1011300052E4C301B2010E94F33820E030E040E7FE
:1011400052E40E94F338F8016083718382839383B1
:10115000CEC0E15CFD4F77FA709477F87094DECFE3
:101160008F5F0A3008F4D1C0843009F4CEC00A5031
:10117000C2CFC301B2010E94D6390E94143710E0D9
:101180000132110508F0C1C0F801EF5AFF4F0C946D
:101190003E3A633008F4BCC060934B02A8C0609331
:1011A0004E02A5C060934C0202C060934D020E94A3
:1011B00020329DC080916002662311F0846095C04A
:1011C0008B7F93C080916002662311F080648DC094
:1011D0008F7B8BC080916002662311F0806801C014
:1011E0008F778093600280E00E94EC2B80C0609338
:1011F0004F027DC0409250025092510260925202C2
:101200007092530274C04092540250925502609200
:101210005602709257026BC080916002662311F0F3
:10122000816001C08E7F809360020E949E2B5FC010
:1012300080916002662321F084FF6DC0806255C0FA
:101240008F7D53C080916002662311F0886001C0D9
:10125000877F809360020E940C3149C080916002B8
:10126000662311F0806141C08F7C3FC060936102B2
:101270003EC0409262025092630260926402709299
:10128000650235C040926602509267026092680221
:10129000709269022CC070E070936B0260936A02D6
:1012A00026C040926C0250926D0260926E02709263
:1012B0006F021DC0409258025092590260925A0229
:1012C00070925B0208C040925C0250925D02609294
:1012D0005E0270925F020E94CF0109C0809160029D
:1012E000662311F0826001C08D7F809360020E94AE
:1012F000C51D13C055E0F52E10C048E0F42E0DC0FA
:10130000F82E0BC034E0F32E08C023E0F22E05C007
:1013100096E0F92E02C08AE0F82E8F2D08C0809149
:101320000A02817211F089E0E7CB0E94C9090E948C
:10133000172DE4CB002329F0893209F0E1CB0D7F92
:10134000DFCB813208F4DCCB8F3209F4D9CB883281
:1013500089F08B3389F01F3488F4212F30E01F5F30
:101360009FE9980FF901EF5EF84F9A3108F4805227
:101370008083C6CB02E0C4CB04E0C2CB01E0C0CB8B
:1013800087E00E940B2D8FEF0E94E61D0E94812DA9
:10139000CACA2F923F924F925F926F927F928F9222
:1013A0009F92AF92BF92CF92DF92EF92FF920F93F4
:1013B0001F93CF93DF93CDB7DEB7CA54D1090FB6D1
:1013C000F894DEBF0FBECDBF8AE3E0EBF2E0DF01B1
:1013D0001D928A95E9F78BE0E0E7F2E0A1EBB2E03D
:1013E00001900D928A95E1F780911107843211F0F6
:1013F0000C94531781E08093B1021092B20283E003
:101400008A8FB1E0BBA3212C312C1CA61BA610E0B7
:101410001B8E1F8EEE24E394F12CEAE0AE2EB12C4D
:10142000F1E68F2EF3E09F2E8A8DE82FF0E0EF5E3D
:10143000F84FD080DD2009F437C29FEB9D0D9A3123
:1014400010F00C9422178F5F8A8FBE016A5E7F4F67
:10145000CE014A960E94E734882311F40C94241795
:101460004E885F88688C798CC301B2010E94D6399E
:101470000E941437062F70E080E090E00E9445370C
:101480009B01AC01C301B2010E949B3520E030E01A
:1014900048EC52E40E94F3380E9460390E941437ED
:1014A000CB01E7E4DE1629F0FDE4DF1609F4EAC01B
:1014B00035C1083209F4C6C020F5043168F40131A1
:1014C00008F08AC0043009F452C008F464C00A303D
:1014D00009F445C00C9432170C3109F440C050F4A3
:1014E000063110F00C94321725E1201B2093B30233
:1014F00026E0ADC00E3199F1063209F44CC00C94CF
:1015000032170D3309F498C0A8F4053381F140F483
:101510000B3209F47AC0013309F477C00C94321706
:101520000C3310F00C9432176AEC600F6093B70222
:1015300029E08DC00C3538F40A3508F053C0003569
:1015400081F10C9432170C3551F00F3510F00C94DA
:1015500032172EE5201B2093B20225E078C00097B9
:1015600031F42F8D21110C94261731E03F8F009319
:10157000B002202F2D7F2C3119F00C3509F064C0FA
:10158000009721F00A9711F00C943217600F6093C6
:10159000B00220E061C04F8D41110C942617A2E0EB
:1015A000AF8F0093B102063209F050C0843191052B
:1015B00059F08E31910541F08832910529F082333E
:1015C000910511F00C943217B5010E94083A665744
:1015D0006093B10221E040C06FEE600F6093B502EE
:1015E00022E035C0892B31F466EA600F6093B402C3
:1015F00023E032C06A30710511F00C9432170A35BD
:1016000011F40C94321724E027C0BF8DB1110C9453
:101610002617013331F41092B60228E0E3E0EF8F91
:101620001BC00A9711F00C943217F1E0F093B60248
:1016300028E033E03F8F10C0892B11F00C94321753
:101640002AE00AC027E003C020E001C021E0892B86
:1016500019F087E10C945A17C70102C0880F991F2F
:101660002A95E2F72BA53CA528233923232B19F033
:1016700085E10C945A17ABA5BCA5A82BB92BBCA728
:10168000ABA7D2CE892B29F7063018F4033058F0D7
:1016900016C0083010F40C9432170A30F0F00E31F6
:1016A00059F00C943217002319F0013011F104C0E5
:1016B000B3E0B093B8021DC00093B8021AC0043062
:1016C00021F0053031F080E101C080E28093BA0260
:1016D00002C01092BA028CE00DC0093031F0809146
:1016E000B90280648093B90202C01092B9028DE001
:1016F00001C08BE0F70102C0EE0FFF1F8A95E2F7F1
:101700002BA53CA52E233F23232B09F0B1CF2BA5DE
:101710003CA52E2B3F2B3CA72BA786CE8D2DDD0C79
:10172000990BAA0BBB0BFC01E654F109E531F1055D
:1017300010F00C943217EE58FF4F0C943E3A409242
:10174000BC025092BD026092BE027092BF0280E065
:1017500087C04092C0025092C1026092C202709251
:10176000C302116081E07CC04092C4025092C50265
:101770006092C6027092C702126082E071C040920D
:10178000C8025092C9026092CA027092CB021460E1
:1017900083E066C00093CC0284E062C0C301B20162
:1017A0000E940D376093CD027093CE028093CF02DA
:1017B0009093D00285E054C04092D1025092D20260
:1017C0006092D3027092D40286E04AC04092D50261
:1017D0005092D6026092D7027092D80287E040C041
:1017E0004092D9025092DA026092DB027092DC02DF
:1017F00088E036C020E030E04FE753E4C301B20197
:101800000E94B338181614F40C9428170093DD02C4
:1018100089E026C04092DE025092DF026092E00230
:101820007092E1023B8D31603B8F8AE019C040929B
:10183000E2025092E3026092E4027092E5024B8D64
:1018400042604B8F8BE00CC04092E6025092E70260
:101850006092E8027092E9028B8D84608B8F8CE03D
:101860006701082E02C0CC0CDD1C0A94E2F7960139
:1018700022213321232B11F00C942A17D40102C00A
:10188000B595A7958A95E2F7A0FF0BC020E030E060
:10189000A901C301B2010E94913687FF02C00C94D6
:1018A0002C172C283D28C0CDBB8DBB2329F0EF8DF4
:1018B000E11102C0F2E0FF8F25FE0FC08091CD0242
:1018C0009091CE02A091CF02B091D002813896497A
:1018D000A849B10514F00C942E173BA1332329F02D
:1018E00020FC02C00C94381718C08091B2028130DD
:1018F00071F44F8D4230E1F58091B1028035C1F134
:101900008823B1F120FC02C00C94381731C08091BB
:10191000710281112DC020FE1BC08091B302813065
:1019200039F523E333E34BEC51E46091BC02709151
:10193000BD028091BE029091BF020E94F338609375
:10194000BC027093BD028093BE029093BF0210C090
:1019500080917F0290918002A0918102B0918202D9
:101960008093BC029093BD02A093BE02B093BF02CD
:1019700030FC10C080917B0290917C02A0917D028E
:10198000B0917E028093D9029093DA02A093DB0299
:10199000B093DC028091B002843039F426FC03C09D
:1019A0008CE10C945A17E89426F88091B5028823AC
:1019B00069F0813029F48FAF1DAE92E09BAF0BC070
:1019C0001FAEA2E0ADAFB1E0BBAF05C0E2E0EFAF4C
:1019D000F1E0FDAF1BAE8091B302813021F02F8D7D
:1019E0002330C9F52FC060EBC62E62E0D62EE12C65
:1019F000F12C3B8DA32EB12CC5010E2C02C0959568
:101A000087950A94E2F780FF12C023E333E34BEC9F
:101A100051E4D6019E966D917D918D919C91D197C7
:101A20000E94F338F60166A777A780AB91ABFFEF72
:101A3000EF1AFF0A24E0C20ED11C33E0E316F104D2
:101A4000D9F6CDCF8091B602813029F44B8D443048
:101A500011F00C9430178CE0E4E9F2E0DE0111960D
:101A600001900D928A95E1F78BA59CA591FD08C088
:101A70000091B0020A30C9F00C3509F4B3C01EC1A0
:101A80008091B702873018F08DE10C945A1790912D
:101A90007602891769F3BE016F5F7F4F0E948F1E28
:101AA000882311F40C944617E3CF9B8D911103C04A
:101AB0008AE10C945A17C10180759927892B09F482
:101AC0006FCF6091D1027091D2028091D302909138
:101AD000D4020E94D6390E9414376730A8F680914C
:101AE000CC02843141F0823011F00C94321727FE81
:101AF00002C00C943217AFEA2A22662319F0615013
:101B000069A703C0B091B702B9A760EC72E089A5DC
:101B10000E948F1E882311F40C9446170091CC026A
:101B20004090AC025090AD026090AE027090AF0257
:101B300040EBE42E42E0F42E50E7A52E52E0B52E05
:101B4000C12CD12CEB8D8E2E912CC4010C2C02C0FB
:101B5000959587950A94E2F780FF35C0043151F5D9
:101B6000D501D0962D913D914D915C91D39758968A
:101B70006D917D918D919C915B970E949B35F701B2
:101B800026A537A540A951A90E949B35D70150969B
:101B90006D937D938D939C935397B2E0CB1213C0BA
:101BA000A30192010E949B35F701608B718B828BA0
:101BB000938B09C0F70186A597A5A0A9B1A9808B31
:101BC000918BA28BB38BFFEFCF1ADF0A24E0E20EDA
:101BD000F11C34E0A30EB11C43E0C416D10409F09B
:101BE000B4CF3FC18B8D882309F462CF4090AC0203
:101BF0005090AD026090AE027090AF0220E7822E4E
:101C000022E0922EDE0111967D0130EBC32E32E0F0
:101C1000D32EA12CB12CE82FF0E0F8A7EFA38FA1D1
:101C200098A50A2C02C0959587950A94E2F780FF43
:101C300029C0D7012D913D914D915C91F401608DAA
:101C4000718D828D938D0E949B35D6019E962D912C
:101C50003D914D915C91D1970E949B35F60166A70D
:101C600077A780AB91ABF2E0AF1216C0A30192014F
:101C70000E949B35D6019E966D937D938D939C9388
:101C8000D1970AC0F40180A991A9A2A9B3A9F6012C
:101C900086A797A7A0ABB1ABFFEFAF1ABF0A24E0AE
:101CA000820E911C34E0E30EF11C44E0C40ED11C02
:101CB00083E0A816B10409F0B2CFD2C09F8D933053
:101CC00069F40E3109F494C0053309F4C3C00C3132
:101CD00009F0C6C060EC72E086E08DC0AB8DAA232F
:101CE00081F3B091B402BFA34090AC025090AD021A
:101CF0006090AE027090AF0280E7A82E82E0B82E0E
:101D000090EBE92E92E0F92EFE0131964F01C12CA5
:101D1000D12C2A2F30E03AA729A789A59AA50C2C07
:101D200002C0959587950A94E2F780FD0BC0F501F6
:101D3000808D918DA28DB38DF70186A797A7A0AB5B
:101D4000B1AB44C0053309F441C0FFA1F1112BC070
:101D5000D501D0962D913D914D915C91D397F40191
:101D600060817181828193810E949C35D7019E960A
:101D70002D913D914D915C91D1970E949C35F70139
:101D800066A777A780AB91ABF2E0CF121FC0A3018B
:101D900092010E949C35D7019E966D937D938D9301
:101DA0009C93D19713C0F501208D318D428D538DB9
:101DB000D7019E966D917D918D919C91D1970E94B6
:101DC0009C35F70166A777A780AB91ABFFEFCF1AE1
:101DD000DF0A24E0A20EB11C34E0E30EF11C44E063
:101DE000840E911C83E0C816D10409F096CF69CF08
:101DF00060EC72E087E00E948F1E882311F40C943F
:101E000046179B8D911103C019A61F8E2AC0A0E70B
:101E1000B2E0E0EBF2E080E090E04B8D242F30E088
:101E2000A901082E02C0559547950A94E2F740FD96
:101E30000AC058964D915D916D917C915B97408B56
:101E4000518B628B738B0196149634968330910577
:101E500039F706C08091B102823010F00C9434172B
:101E600019A68091B1028FA3803529F49B8D911121
:101E70000C9436177AC2AF8DA23009F076C2BFA19A
:101E8000B11104C0EB8DE11170C22AC020E030E036
:101E9000A9016091BC027091BD028091BE02909137
:101EA000BF020E949136882309F4E2C7FFA1FC38E3
:101EB00009F445C240F4F230A9F0F330B1F0F1304A
:101EC00009F053C20AC02FA12E3809F438C208F411
:101ED00033C22F3809F430C248C23B8D311145C29C
:101EE0001F8E43C24BA144604BA38B8D882309F402
:101EF000DFCDBBADAB2FB0E0B8ABAFA7FDADEF2FE3
:101F0000F0E0FCABEBAB81E090E07C010BAC02C0FD
:101F1000EE0CFF1C0A94E2F70DAC02C0880F991F6B
:101F20000A94E2F7E82AF92A2B8D822F90E08E217D
:101F30009F21892B09F49EC7FD01EE0FFF1FEE0FB5
:101F4000FF1FE055FD4FAA0FBB1FAA0FBB1FA857CD
:101F5000BD4F2D913D914D915C9166A577A580A9CE
:101F600091A90E949B352B013C01EBA9FCA9EE0F26
:101F7000FF1FEE0FFF1FE055FD4FABA9BCA9AA0F35
:101F8000BB1FAA0FBB1FA857BD4F2D913D914D916F
:101F90005C9166A577A580A991A90E949B354B010C
:101FA0005C01610130E8C322DD2427FEF5C0E8941E
:101FB00027F84CE050E06EED72E088E892E00E9475
:101FC0005E3A892B11F481E275C78091B3028130AA
:101FD000B1F423E333E34BEC51E46091D50270910B
:101FE000D6028091D7029091D8020E94F338609374
:101FF000D5027093D6028093D7029093D802809135
:10200000D5029091D602A091D702B091D8028FABA1
:1020100098AFA9AFBAAFA3019201C301B2010E9468
:10202000F33827966CAF7DAF8EAF9FAF2797A50192
:102030009401C501B4010E94F3382B966CAF7DAFBB
:102040008EAF9FAF2B9720E030E040E850E46FA9BF
:1020500078AD89AD9AAD0E94F3382FA938AD49AD5E
:102060005AAD0E94F33827962CAD3DAD4EAD5FAD15
:1020700027970E949B352B962CAD3DAD4EAD5FADA5
:102080002B970E949B356B017C0120E030E0A90179
:102090000E94913687FDF0C6C701B6010E949239B1
:1020A0006B017C012B962CAD3DAD4EAD5FAD2B97FA
:1020B00027966CAD7DAD8EAD9FAD27970E949C3568
:1020C0000E9492399B01AC01C701B60190580E9451
:1020D0009B366B017C019FA1933021F4F7FAF094B9
:1020E000F7F8F09420E030E0A9016FA978AD89AD50
:1020F0009AAD0E94913687FF11C0F7FAF094F7F875
:10210000F0948FA998ADA9ADBAADB0588093D5021F
:102110009093D602A093D702B093D8020FA518A926
:10212000000F111F000F111F00541D4FA701960132
:10213000C501B4010E94F3389B01AC01C301B20197
:102140000E949B3520E030E040E05FE30E94F338DE
:10215000D8016D937D938D939C9313970BA91CA924
:10216000000F111F000F111F00541D4FA7019601F2
:10217000C301B2010E94F338A50194010E949C356D
:1021800020E030E040E05FE30E94F338F801608334
:10219000718382839383E9C0212F30E038AF2FAB66
:1021A000E222F322EF2809F469C631EF232280915D
:1021B000B302813009F47BC0EFA5F8A9EE0FFF1F31
:1021C000EE0FFF1FE054FD4FC080D180E280F3800E
:1021D000A7019601C301B2010E949B352B013C016E
:1021E000EBA9FCA9EE0FFF1FEE0FFF1FE054FD4F00
:1021F00080819181A281B3818FA798ABA9ABBAAB43
:102200009C01AD01C501B4010E949B354B015C01ED
:10221000A3019201C301B2010E94F3382B013C01DA
:10222000A5019401C501B4010E94F3389B01AC01E2
:10223000C301B2010E949C350E9492394B015C019E
:10224000A7019601C701B6010E94F3386B017C011A
:102250002FA538A949A95AA9CA01B9010E94F33882
:102260009B01AC01C701B6010E949C350E949239C6
:102270006B017C016093D5027093D6028093D702E4
:102280009093D8029B01AC01C501B4010E949B351B
:102290004B015C01E894B7F82AE037ED43EA5BE3D1
:1022A000C501B4010E94B33818164CF15EC000EBB2
:1022B00012E08FA998AD0C2C02C0959587950A94D1
:1022C000E2F780FF12C023E333E34BEC51E4D80183
:1022D00050966D917D918D919C9153970E94F3380A
:1022E000F801608B718B828B938BFFEFCF1ADF0A23
:1022F0000C5F1F4F23E0C216D104D9F65DCF20E05A
:1023000030E040E05FE3C501B4010E94B338181625
:102310000CF459CE2FE632E143E85AE3C701B60187
:102320000E94F3389B01AC01C501B4010E94B3388F
:1023300018160CF448CE19C03BA130613BA38FA105
:102340008E58823018F44BA148604BA38B8D8823A4
:1023500009F4AECB4CE050E06EED72E088E892E01C
:102360000E945E3A892B09F42ECE2BA121709BA1ED
:1023700090FF03C0C1018E7D03C0C1018E7D9C7F93
:10238000AF8DA111937E892B09F07AC58E01035F71
:102390001F4F89E0F80111928A95E9F7222309F489
:1023A0004BC08BA59CA5867B892B09F06BC58091C2
:1023B000B002853311F0811165C580917B02909147
:1023C0007C02A0917D02B0917E02898B9A8BAB8BAF
:1023D000BC8B9091790280917802892B4091BC024C
:1023E0005091BD026091BE027091BF024D875E8721
:1023F0006F87788B84608D8B8091600285FF06C02B
:102400008EED92E00E94272B81113EC5B8018EED22
:1024100092E00E94050480910A02811139C50E9450
:10242000671D892B09F434C580E280930A020E945B
:10243000B01E0E94CF342CC580916002F0907902CA
:1024400081FF26C08FA18150833018F0FBA1F0647A
:10245000FBA32B8D222339F03F8D323021F44BA189
:1024600040684BA315C080E1F81212C08091700241
:1024700081509BA19074833030F4992349F09BA143
:1024800090629BA305C0911103C0ABA1A062ABA356
:102490008091CD029091CE02A091CF02B091D00256
:1024A0008093840290938502A0938602B093870262
:1024B0008091B20280937102882311F088E08D8BA5
:1024C0008091BC029091BD02A091BE02B091BF026A
:1024D00080937F0290938002A0938102B093820246
:1024E0008D879E87AF87B88B8090D9029090DA0253
:1024F000A090DB02B090DC02A501940160917B0208
:1025000070917C0280917D0290917E020E949136B2
:10251000BBA1B074EB2E811103C0EBA1E5FF20C07D
:10252000FF2071F0FBA1F7FD0BC0EE2021F040E091
:1025300050E0BA0102C0B501A4018F2D0E943B03F7
:102540008091D9029091DA02A091DB02B091DC0275
:1025500080937B0290937C02A0937D02B0937E02D5
:10256000E1100CC080917B0290917C02A0917D02D1
:10257000B0917E02898B9A8BAB8BBC8B8091DD02F4
:10258000809383028091BA0290917902981751F05A
:1025900049895A896B897C890E943B038091BA02E0
:1025A000809379029D8980917902892B8D8BF0909F
:1025B000B902809178028F1569F080910A02823009
:1025C00029F00E9402028F2D0E9459028091B902C7
:1025D000809378029D8980917802892B8D8B8091E0
:1025E000B002843099F4C090D102D090D202E09031
:1025F000D302F090D40280910A02823039F00E9416
:10260000020240E0C701B6010E94E0318091B502AC
:10261000809374028091B302809372022F8D2330D5
:1026200071F58091B60280937502811108C01092F5
:10263000E6021092E7021092E8021092E902C090BE
:10264000E602D090E702E090E802F090E902A701EC
:1026500096016091AC027091AD028091AE029091B2
:10266000AF020E949136882351F0C092AC02D09202
:10267000AD02E092AE02F092AF020E949E2B8091DA
:10268000B70290917602981769F0809376028CE0F9
:10269000FE013196A4E9B2E001900D928A95E1F72E
:1026A0000E949E2B8091B402809373028091B002AD
:1026B0008632F1F138F48C3109F18E31F9F08A303B
:1026C00069F04FC08C35D1F1863609F441C08832AB
:1026D00009F047C068E872E087E02DC060EC72E066
:1026E00089A50E94D21D8091760239A5381339C080
:1026F0008CE0E0ECF2E0A4E9B2E025C08D898160D5
:102700008D8B4F8D442329F0B8018EED92E00E940D
:102710000504B80180EC92E00E9405048CE0E0EC36
:10272000F2E0A8E8B2E001900D928A95E1F719C0B5
:1027300068E872E086E00E94D21D13C08CE0EEEDE6
:10274000F2E0A0EAB2E001900D928A95E1F707C0AD
:102750008CE0E0EAF2E0DF011D928A95E9F70E9441
:102760009E2B8091B10280937002803509F41CC3C6
:10277000BF8DB23009F018C3813021F4BE01635F10
:102780007F4F06C0811109C08D8981608D8BB80192
:102790008EED92E00E940504FEC28250823008F065
:1027A00093C28091D5029091D602A091D702B091A8
:1027B000D8028F8F98A3A9A3BAA3ABAD94E0A99F29
:1027C00070011124F701E857FD4FF8A7EFA3970117
:1027D00020543D4F3AA729A7D9014D905D906D90A7
:1027E0007C902081318142815381C301B2010E94DA
:1027F0009C356BA77CA78DA79EA7EDADB4E0EB9FA2
:1028000080011124980128573D4F3CAF2BAFC801E0
:1028100080549D4F9EAF8DAFDC018D909D90AD900B
:10282000BC90F9012081318142815381C501B401FD
:102830000E949C356FA778AB89AB9AAB77FA7094FE
:1028400077F87094D501C401B0588B8F9C8FAD8FF1
:10285000BE8FF701E252FD4F2BA53CA54DA55EA50D
:1028600060817181828193810E949B356B017C0123
:10287000F801E252FD4F2FA538A949A95AA9608154
:102880007181828193810E949B354B015C01A7017C
:102890009601C301B2010E94F3386BAB7CAB8DABE8
:1028A0009EABA50194016B8D7C8D8D8D9E8D0E94BC
:1028B000F3389B01AC016BA97CA98DA99EA90E944C
:1028C0009C356BAB7CAB8DAB9EABA5019401C3017A
:1028D000B2010E94F3384B015C01A70196016B8D98
:1028E0007C8D8D8D9E8D0E94F3389B01AC01C501BE
:1028F000B4010E949B352BA93CA94DA95EA90E9459
:102900001B366B017C019BA192FF13C02DEB37E3BB
:1029100046E055EBC701B6010E94B33887FD1DC0E4
:102920002BED3FE049EC50E4C701B6010E949B3516
:1029300012C02DEB37E346E055E3C701B6010E9414
:102940009136181654F02BED3FE049EC50E4C701E6
:10295000B6010E949C356B017C01809054029090DE
:102960005502A0905602B09057022F8D38A149A170
:102970005AA1CA01B9010E949C35A50194010E9487
:102980009B35A50194010E94F3380E9492394B01B6
:102990005C0120E030E040E05FE3C701B6010E9447
:1029A000F3382F8D38A149A15AA10E94F3389F779F
:1029B000A50194010E949B360E9480370E94143723
:1029C0007CAB6BABDB01AB2B09F4D8CE1D894B0183
:1029D000A12CB12C13FF12C0C501B4010E944337D2
:1029E0009B01AC016D857E858F8598890E94F338A7
:1029F0006D877E878F87988B177F1D8BC501B401EC
:102A00000E9443374B015C019B01AC01C701B60139
:102A10000E949B366BA37CA38DA39EA3EFADB4E075
:102A2000EB9FC00111248C0108571D4FFC01E2529D
:102A3000FD4FD8012D913D914D915C916081718147
:102A4000828193810E949B35A50194010E949B364F
:102A500027966CAF7DAF8EAF9FAF27972BA13CA180
:102A60004DA15EA1CA01B9010E94F3389B01AC01DE
:102A700060E070E080E090E40E949B356B017C0197
:102A80002BEA3AEA4AE25EE36BA17CA18DA19EA10A
:102A90000E94F3384B015C0120E030E040E850E454
:102AA000C701B6010E949C359B01AC01C501B40170
:102AB0000E94F3386FAB78AF89AF9AAF20E030E077
:102AC00040E05FE3C701B6010E94F33823966CAF84
:102AD0007DAF8EAF9FAF23971F8E22242394312C7E
:102AE000EBA9FCA9E215F30509F448CEBF8DBC3073
:102AF00008F044C02B8D3C8D4D8D5E8D23966CADC2
:102B00007DAD8EAD9FAD23970E94F3386B017C01A4
:102B1000A30192016FA978AD89AD9AAD0E94F338F7
:102B2000A70196010E949C357B016C01A3019201D3
:102B300023966CAD7DAD8EAD9FAD23970E94F3388B
:102B40004B015C012B8D3C8D4D8D5E8D6FA978AD59
:102B500089AD9AAD0E94F3389B01AC01C501B40167
:102B60000E949B352B013C01EF8DEF5FEF8F4701FA
:102B700056018B8E9C8EAD8EBE8E65C0B10180E0FD
:102B800090E00E9443372BA13CA14DA15EA10E9481
:102B9000F3386B017C010E9496366B8F7C8F8D8F92
:102BA0009E8FC701B6010E9484394B015C01A9A523
:102BB000BAA5CD90DD90ED90FC90F7FAF094F7F87F
:102BC000F094ADADBEAD8D919D910D90BC91A02DB9
:102BD0008F8F98A3A9A3BAA3A70196016B8D7C8DB3
:102BE0008D8D9E8D0E94F3382B013C012F8D38A1D5
:102BF00049A15AA1C501B4010E94F3389B01AC015F
:102C0000C301B2010E949C352B013C01A701960132
:102C1000C501B4010E94F3386B017C012F8D38A1EE
:102C200049A15AA16B8D7C8D8D8D9E8D0E94F338AC
:102C30009B01AC01C701B6010E949B356B8F7C8F55
:102C40008D8F9E8F1F8EA30192016BA57CA58DA5F4
:102C50009EA50E949C35EFA1F8A5608371838283B5
:102C600093832B8D3C8D4D8D5E8D6FA578A989A9A1
:102C70009AA90E949C35ABADBCAD6D937D938D93AD
:102C80009C93139727962CAD3DAD4EAD5FAD279726
:102C9000F80160817181828193810E949C35D80105
:102CA0006D937D938D939C931397BE01635F7F4FCC
:102CB00088E892E00E94050480910B0281116BC0AC
:102CC000BFEF2B1A3B0A0CCF8D8984608D8B8091CE
:102CD0000A02823009F45FC00E94020280910B0256
:102CE000811162C0FBA1F071FF2E10920F022BA187
:102CF00023FB882780F90E94EC2B86B1807290918B
:102D0000F001891749F084E00E940E2B0E94B61B47
:102D100080E00E94EC2B48C0B8018EED92E00E944A
:102D2000050481E08093090282E00E941E2B0E942C
:102D3000B61B80910B02811137C080910A0281116C
:102D4000F6CF80910902813081F4FF2051F08CE0B0
:102D5000E1EFF1E0ADEFB1E001900D928A95E1F77E
:102D600007C085E00E940E2B03C081E080930F0214
:102D70001092090280E00E94EC2B0E94B61B0E9478
:102D80009A2A0E94771D0E940F320E94982E8091ED
:102D90000F0281118CC08CE0EEEDF2E0A8E8B2E009
:102DA00001900D928A95E1F78091B80280937702A5
:102DB000882309F47FC00E940202809177029091DB
:102DC0000A02833041F49230D1F188E00E941E2B38
:102DD0000E94B61B34C081E080937002109274028E
:102DE0001092730210927102109276021092790280
:102DF0001092780284E680931102809312028093ED
:102E00001302923091F064E972E080E00E948F1E1C
:102E10008823E1F10E949E2B40E050E0BA0180E05F
:102E20000E94100380E00E94590283EA92E00E940F
:102E3000F82C8AE392E00E94F82C0E94932E1092C4
:102E400077022FC081E036C082E034C088E132C012
:102E500086E230C089E12EC084E02CC08BE12AC01C
:102E600085E228C084E126C08EE124C08FE122C023
:102E700086E120C080E21EC082E21CC083E21AC04C
:102E800084E218C080E116C08FE014C087E012C051
:102E90008CE0EEEDF2E0A8E8B2E001900D928A95A8
:102EA000E1F780E007C01A8E1BA20C94030A0E946F
:102EB00059037ACFC65BDF4F0FB6F894DEBF0FBE63
:102EC000CDBFDF91CF911F910F91FF90EF90DF90D9
:102ED000CF90BF90AF909F908F907F906F905F90BA
:102EE0004F903F902F9008953F924F925F926F9234
:102EF0007F928F929F92AF92BF92CF92DF92EF928A
:102F0000FF920F931F93CF93DF93CDB7DEB7A497B4
:102F10000FB6F894DEBF0FBECDBF10910E07112380
:102F200091F181E080930A0289EA92E00E94F82CF4
:102F3000812F0E94D22C0E94072D85EF91E00197EE
:102F400039F0EFE9FFE03197F1F700C00000F7CF6B
:102F50001150123030F08FB7F89410920E078FBFD7
:102F600012C083EA92E00E94F82C81E992E00E946C
:102F7000F82C0E94932E80E10E94142B80910D0763
:102F800084FFFCCFE8CF10910D07112309F4BBC2D9
:102F900014FF04C081E080930B02D0C310FFBFC1B7
:102FA0008CE0E1EFF1E0DE01599601900D928A95F7
:102FB000E1F7BE01675E7F4FCE010D960E94622B46
:102FC0008CE30E943D0280910A028830E1F058F4BF
:102FD000813099F1A8F0823099F1843009F043C032
:102FE00084EF92E03EC0803229F118F4803171F014
:102FF0003AC0803441F18038B1F58CED92E031C0B7
:1030000087E093E02EC083E093E02BC080910C0218
:1030100087FD10C08DEF92E00E94F82C80910C0289
:1030200080FF06C080E31AC082FF17C085FFFACF79
:1030300081E314C089EF92E014C08EEE92E011C0DB
:1030400088EE92E00EC082EE92E00E94F82C809111
:103050000C0283FFE9CF83E301C082E30E943D02BB
:1030600002C00E94F82C80914F02F82FF170BF2E01
:1030700080FF07C080911602882319F085ED92E049
:1030800053C04090AC025090AD026090AE02709080
:10309000AF0254E9852E52E0952E9E012F5F3F4FDF
:1030A0007901CE010D966C0100E0F40161917191FE
:1030B000819191914F0120853185428553850E94F0
:1030C0009C35F7016083718382839383023061F4BE
:1030D000A30192010E949C35F70160837183828372
:1030E0009383BB2019F0CACFB11011C0F701208122
:1030F000318142815381F6016081718182819381A6
:103100000E949B35F60160837183828393830F5FF6
:10311000F4E0EF0EF11C24E0C20ED11C033029F6BE
:10312000B110ACCF8EEC92E00E94F82CCE010D963F
:103130000E94B92C80914F0281FF1FC089EC92E060
:103140000E94F82C9091EB068091CA03981710F01A
:10315000815F01C08150891B0E94D22C8CE20E94A9
:103160003D028091EB029091EA02981710F080588E
:1031700001C08150891B0E94D22C84EC92E00E94F5
:10318000F82C80910A028C7749F06091AF0370911E
:10319000B0038091B1039091B20303C060E070E08E
:1031A000CB010E949B2C8CE20E943D026091170291
:1031B000709118028091190290911A0240E00E94C9
:1031C000FE2B0E94F12EF82E0E94A32B082F86B111
:1031D000982F90728091F001E92EE8268F2D802B98
:1031E0008E2959F18FEB92E00E94F82CEE2019F015
:1031F00080E50E943D02FF2079F0F0FE03C088E5E3
:103200000E943D02F1FE03C089E50E943D02F2FEEC
:1032100003C08AE50E943D02002379F000FF03C04D
:1032200082E50E943D0201FF03C088E40E943D0246
:1032300002FF03C083E50E943D02809116028823AD
:1032400021F081508093160218C080910A028C7779
:1032500011F08DE101C089E0809316028091150282
:10326000811103C081E08093150289EB92E00E94F6
:10327000F82CCE0101960E94B92C00911502002372
:1032800021F001500093150242C080910A028C7710
:1032900011F083E101C089E08093150284EB92E094
:1032A0000E94F82C809111020E94D22C8CE20E9484
:1032B0003D02809112020E94D22C8CE20E943D02BB
:1032C000809113020E94D22C8091B00087FF05C02C
:1032D0002D9B02C002E001C001E0439B03C040E41B
:1032E000F42E03C0002399F0F12C80EB92E00E94B1
:1032F000F82C002339F0013011F483E501C083E498
:103300000E943D02FF2019F086E40E943D028EE3F8
:103310000E943D020E94072D81E00E94142B812F04
:10332000887E09F467C080910A02982F937009F093
:1033300050C08872A1F080910C02807C81F40E94C0
:103340006E2682E080930E0280910A02803239F468
:1033500017FDF2C180910C02806880930C0280916D
:103360000A02811103C091E090930C0216FF07C07E
:1033700085FD05C090910C02906490930C0213FFA0
:1033800005C0807E19F480E180930A0215FF21C0F8
:1033900083EA92E00E94F82C8FE492E00E94F82CDD
:1033A0000E94932E80910C0287FD0EC090910A021C
:1033B000903439F483FFBCC1837E826080930C0219
:1033C000B7C1903809F0B4C180910C02806280933B
:1033D0000C0217FF0CC080910A02813029F4809101
:1033E0000C02856080930C0280E880930A0288EECC
:1033F0000E94142B11FF44C0812F8876F1F5809133
:103400000A02803471F480910C0285FD0AC084FFA9
:1034100003C010920A0205C082FF03C08860809337
:103420000C0280910A02882381F084FF26C09091CB
:103430000C0290FF22C0803141F480911402882355
:1034400021F088608093140218C010920E020E942E
:10345000671D892B71F080910C0286FD0AC01092C5
:103460000C0288E080930A020E94B01E0E94CF34B2
:1034700004C010920C0210920A0282E00E94142BE7
:1034800012FF41C080910A02807D90910C02882336
:10349000D9F080910D02811117C097FD15C00E94CF
:1034A0006E268091CA038093C8030E949226809161
:1034B0000E0281FF05C090910C02916090930C0266
:1034C000897F80930E021CC097FF0AC010920E02E3
:1034D0000E94771D0E949A2A0E9459030E940F326F
:1034E00080910C0285FF08C08F77816080930C0269
:1034F00080E480930A0204C010920C0210920A0227
:1035000084E00E94142B90910F07992309F4ABC01B
:103510008FB7F89410920F078FBF4091110290FD62
:1035200002C0842F01C084E691FD865F92FD8A501F
:1035300093FD8F5F94FD8150893C08F088EC8A30C0
:1035400008F48AE03091120295FD02C0232F01C0D9
:1035500024E696FD22E397FD29E1481303C02317D3
:1035600009F481C080931102209312021092150277
:103570001091CA033090EB0689E9D82E96E7E92E20
:1035800026E9F22E0EE732E3432E131509F457C055
:10359000812E912C489CC001499C900D1124FC0166
:1035A000E553FC4F5F01CF010E94F41C562E672E9D
:1035B000782EC92E2D2D3E2D4F2D502F0E94B33821
:1035C00018164CF42D2D3E2D4F2D502F6D2D7E2D88
:1035D0008F2D902F08C0252D362D472D5C2D652D64
:1035E000762D872D9C2D0E94F338F501668B778B05
:1035F000808F918F489CC001499C900D11249C01A3
:1036000025533C4F7901F90182A093A0A4A0B5A055
:10361000A501940166897789808D918D0E94B338C8
:1036200018162CF4F701868A978AA08EB18E1F5F38
:10363000103109F410E0D52C73010C2DA6CF8D2D7F
:103640009E2DAF2DB02F8093090790930A07A0936A
:103650000B07B0930C070E946E268091CA038093DB
:10366000C8030E94922610911007112309F459C033
:103670008FB7F894109210078FBF9091130210FD2E
:1036800002C0892F01C084E611FD865F12FD8A50B9
:1036900013FD8F5F14FD8150893C08F088EC8A305F
:1036A00008F48AE09817D1F08093130280910A02FF
:1036B00081110DC040917B0250917C0260917D028E
:1036C00070917E02809179020E94100305C0809162
:1036D0000E02886080930E021092150280910A02F9
:1036E00015FF0DC0803159F490911402911102C060
:1036F00092E003C090FF03C0946090931402107C8A
:1037000081F0882311F0887361F01091780216FF20
:1037100002C01F7B01C01064812F0E9459021093C8
:10372000780280910A028C7F49F00E94B01E06C088
:1037300080E480930A0248CE80E218CEA4960FB6A9
:10374000F894DEBF0FBECDBFDF91CF911F910F91D7
:10375000FF90EF90DF90CF90BF90AF909F908F90B1
:103760007F906F905F904F903F900895CF92DF923F
:10377000EF92FF921F93CF93DF930E947417809173
:103780000C02882309F4FEC00E94671D009771F4A3
:10379000C091790280917802C82BC0907B02D090B2
:1037A0007C02E0907D02F0907E020EC0FC01C18997
:1037B000C073439B02C020E401C020E0C22BFC0187
:1037C000C6A4D7A4E0A8F1A88091600281FF03C03D
:1037D00080E20E94FC2ADC2FD07311E0C07C809133
:1037E0000C02882309F4CEC090910B029111CAC03B
:1037F00080FFC5C090910A02292F207C09F474C073
:1038000082FD12C01092140240E050E0BA0180E044
:103810000E94100380E00E94590280910C028D7F6B
:10382000846080930C02ABC09038E1F483EA92E0AC
:103830000E94F82C8CE092E00E94F82C0E94932EBB
:1038400040E050E0BA0180E00E94100380E00E9456
:1038500059020E94513280910B02811193C00E9443
:103860007417F9CF903419F48F7D80930C028091F6
:103870000C0283FF84C0909179029923C1F081FDED
:1038800016C08091600281FF06C080910E028860A0
:1038900080930E020CC0B701A6018D2F0E94100369
:1038A00041E060E070E080E890E40E94E0318091C7
:1038B0007802882371F080910C0281FD0AC08C2F60
:1038C0000E94590241E060E070E080E89FE30E94BE
:1038D000E03180910C0281FD52C0806180930C0226
:1038E00082E00E941E2B4BC0809114028823C9F1F4
:1038F00081FF0DC0809179028823B1F040E050E053
:10390000BA0180E00E9410031093140238C08C703A
:10391000B1F18091790281110AC08091140283FF74
:1039200003C082E00E941E2B1092140228C083EA7A
:1039300092E00E94F82C85E192E00E94F82C0E940F
:10394000932E8091600281FF06C080910E028860F4
:1039500080930E02E2CFB701A6018D2F0E941003C3
:10396000DCCF80910E0283FF0AC0B701A6018D2F24
:103970000E94100380910E02877F80930E020E94A6
:1039800074172DCFDF91CF911F91FF90EF90DF90B3
:10399000CF9008950E94671D892B19F082E00C9446
:1039A0001E2B0895F894F999FECF92BD81BD81E058
:1039B0008FBB80B58627482F082E000C550B262F6D
:1039C00030E024233523232B39F06F3F19F060BDFD
:1039D00084E006C084E104C0882321F060BD84E255
:1039E0008FBBF99A78940895BF92CF92DF92EF92AD
:1039F000FF920F931F93CF93DF937C01FC0102A5ED
:103A000013A5D4A5C5A5818980FF18C060911202B5
:103A100070E080E090E00E9445372AE037ED43E215
:103A20005CE30E94F3389B01AC01B8018D2F9C2F01
:103A30000E94F3388B01D82FC92F2DC082FD17C0EB
:103A40006091110270E080E090E00E9445372AE02A
:103A500037ED43E25CE30E94F3389B01AC01B8010F
:103A60008D2F9C2F0E94F3388B01D82FC92FF7017F
:103A7000B6A0C7A0D0A4F1A42B2D3C2D4D2D5F2DB9
:103A8000B8018D2F9C2F0E94B338181624F40B2DEB
:103A90001C2DDD2DCF2D20E030E040E85FE3B801A4
:103AA0008D2F9C2F0E94B338181624F000E010E0F0
:103AB000D0E8CFE3B8018D2F9C2FDF91CF911F91DC
:103AC0000F91FF90EF90DF90CF90BF90089580917D
:103AD000CA039091EB06981739F022E3829FC00148
:103AE000112485539C4F089580E090E008958CE167
:103AF000E1EFF6E0DF011D928A95E9F71092CA0323
:103B00001092EB0681E08093C9031092C8030895D8
:103B10009F92AF92BF92CF92DF92EF92FF920F935C
:103B20001F93CF93DF935C018A017B01E40EF51EA6
:103B3000EB01912C6C01C61AD70ACE018C0D9D1D8C
:103B4000CE15DF0589F0911008C0292D990C330B93
:103B5000232F221F2227221F01C021E06991922ECC
:103B6000960E0E94D21CE9CF692DC501800F911FCE
:103B7000DF91CF911F910F91FF90EF90DF90CF9049
:103B8000BF90AF909F900C94D21C6AE080E090E0D0
:103B90000E94D21C45E550E06BE172E081E090E0CC
:103BA0000C94881D0F931F93CF93C82F8B010E94F5
:103BB00002022DE0C29FC00111244CE050E0B80188
:103BC0009E5FCF911F910F910C94881DEF92FF92F1
:103BD0000F931F93CF93DF93CDB7DEB72C970FB61C
:103BE000F894DEBF0FBECDBF182F80FF0BC085E558
:103BF000ECE0F3E0ABE1B2E005900D928A95E1F7DD
:103C00000E94C51D11FF10C0CE0101967C018CE001
:103C1000F70111928A95E9F700E0B701802F0E9421
:103C2000D21D0F5F0830C9F712FF14C060E080E0BA
:103C300093E00E94D21C60E081E093E00E94D21CDD
:103C400060E081E593E00E94D21C60E082E593E0B1
:103C50000E94D21C13FF0AC060E08EEA93E00E942B
:103C6000D21C60E08FEA93E00E94D21C2C960FB623
:103C7000F894DEBF0FBECDBFDF91CF911F910F91A2
:103C8000FF90EF900895F999FECF92BD81BD81E03C
:103C90008FBB80B508959F92AF92BF92CF92DF9273
:103CA000EF92FF920F931F93CF93DF935B018A01F3
:103CB0007C01E40EF51EEC01912C6B01C81AD90AA7
:103CC000C6018C0F9D1FCE15DF0589F00E94431E93
:103CD000911008C0292D990C330B232F221F222766
:103CE000221F01C021E0982E920E8993E9CFC501D1
:103CF000800F911F0E94431E21E030E0981611F0C2
:103D000020E030E0C901DF91CF911F910F91FF902A
:103D1000EF90DF90CF90BF90AF909F9008951F934A
:103D2000CF93DF93182FEB018DE0189FB001112482
:103D30007E5F4CE050E0CE010E944B1E892B59F46F
:103D40008CE0FE0111928A95E9F7BE01812F0E9455
:103D5000D21D80E001C081E0DF91CF911F910895D5
:103D60002F923F924F925F926F927F928F929F928B
:103D7000AF92BF92CF92DF92EF92FF920F931F9379
:103D8000CF93DF93CDB7DEB7EC970FB6F894DEBFD5
:103D90000FBECDBF80910E0280FD87C790911203A8
:103DA0008091EC06981709F480C78091EF069091F6
:103DB000F006892B09F015C310910E0212FF09C0FD
:103DC0008091EB0622E3289FC001112485539C4F6C
:103DD00002C00E94671D9093F0068093EF0620902A
:103DE000EF063090F0062114310409F45EC700910B
:103DF0009903802F817000FF03C010929903EAC0DD
:103E0000909198039F5F953009F0892F80939803D4
:103E1000E82EF12C32E13E9DF0013F9DF00D112482
:103E2000E25CFC4FF093EE06E093ED06D101509674
:103E30009C915097908BE2E18E9FC001112420E06D
:103E400030E04D915D916D917D91F901E80FF91F81
:103E5000E25CFC4F689412F8440F551F661F771FF1
:103E60001694D1F740835183628373832C5F3F4F55
:103E70002C30310531F722E12E9DF0012F9DF00D00
:103E800011249F01225C3C4FF10184859585A68514
:103E9000B78543E0880F991FAA1FBB1F4A95D1F72A
:103EA000F90184879587A687B787D1011C966D9104
:103EB0007D918D919C911F970E94433760939E0343
:103EC00070939F038093A0039093A103F101268D2B
:103ED000378D40A151A10E949B369B01AC0160939C
:103EE000A2037093A3038093A4039093A50360E0BF
:103EF00070E080EA9FE30E949B366093A603709374
:103F0000A7038093A8039093A90310929A03109299
:103F10009B0310929C0310929D0311FD02C003FFAE
:103F20001FC06091B7037091B8038091B90390915D
:103F3000BA036093AF037093B0038093B10390937F
:103F4000B2039B01AC010E94F338D10152966D93EC
:103F50007D938D939C935597077F009399030FC092
:103F6000F10162897389848995890E9492396093ED
:103F7000AF037093B0038093B1039093B203F2E167
:103F8000FE9DC001FF9D900D11249C01225C3C4FC1
:103F90007901D90151961C928091600281FF1AC06B
:103FA000F101818985FF16C022A533A544A555A539
:103FB00060E070E080E89FE30E949B366093C3035B
:103FC0007093C4038093C5039093C603E1E0D701C7
:103FD0005196EC931092AB031092AC031092AD0388
:103FE0001092AE03D1015A962D913D914D915C9165
:103FF0005D9729833A834B835C8360E070E080E0C7
:104000009FE30E949B364B015C01F101468C578C6B
:1040100060A071A011FF4BC0F2E0F093AA03D101A0
:104020005296CD90DD90ED90FC905597A7019601AA
:104030000E94F3389B01AC01C301B2010E949B3581
:104040004B015C0120E030E0A9010E94913687FF1E
:104050001DC029813A814B815C81CA01B9010E944E
:104060009C35A30192010E94F3389B01AC01C7016A
:10407000B6010E949B350E9492396093B7037093FA
:10408000B8038093B9039093BA03A8C18092AB039D
:104090009092AC03A092AD03B092AE031092B7031E
:1040A0001092B8031092B9031092BA0397C11092FC
:1040B000AA034092BB035092BC036092BD0370926E
:1040C000BE0312FF0CC01092B7031092B8031092F7
:1040D000B9031092BA03C12CD12C760124C0E0910F
:1040E000CA03EF5FE03109F4E0E08091EB068E1740
:1040F00059F0B2E3BE9FF0011124E553FC4FC28892
:10410000D388E488F58803C0C12CD12C7601C7017F
:10411000B6010E9492396093B7037093B8038093FD
:10412000B9039093BA03C1010E94F41C698B7A8B86
:104130008B8B9C8B9B01AC010E94F33869877A873B
:104140008B879C87D10152962D913D914D915C9129
:1041500055972D833E834F8358870E94913687FF62
:104160006CC029853A854B855C856D817E818F8108
:1041700098850E949B35A50194010E94F3389B010C
:10418000AC01C301B2010E949B356093BB037093E5
:10419000BC038093BD039093BE0320E030E0A901EF
:1041A0000E94913618163CF1B2E0B093AA0329811F
:1041B0003A814B815C81CA01B9010E949C35A301FF
:1041C00092010E94F3389B01AC016D817E818F8149
:1041D00098850E949B350E9492396093B703709333
:1041E000B8038093B9039093BA03809199038860D0
:1041F00080939903F3C0A701960169857A858B8521
:104200009C850E949B35A50194010E94F338609320
:10421000BF037093C0038093C1039093C2032989A5
:104220003A894B895C892093B3033093B40340935C
:10423000B5035093B60333E0B6C0A70196016D8174
:104240007E818F8198850E949B35A50194010E94F3
:10425000F338A30192010E949C3520E030E040E059
:104260005FE30E94F3386D877E878F87988B20E00D
:1042700030E0A9010E94B33818160CF097C02D85C4
:104280003E854F855889C301B2010E94B338181684
:104290000CF088C0A701960169857A858B859C857D
:1042A0000E949B35A50194010E94F3389B01AC014B
:1042B0006093BF037093C0038093C1039093C203C4
:1042C0006D857E858F8598890E94B3381816CCF548
:1042D00089899A89AB89BC898093B3039093B4038D
:1042E000A093B503B093B6032D813E814F815885CD
:1042F00069857A858B859C850E949136811104C0E1
:1043000091E09093AA036AC02D813E814F81588528
:1043100069857A858B859C850E949B35A5019401D2
:104320000E94F3389B01AC01C301B2010E949B358E
:104330006093BB037093BC038093BD039093BE0353
:104340004DC02D853E854F8558892093BB03309302
:10435000BC034093BD035093BE032093BF0330932F
:10436000C0034093C1035093C20329813A814B811A
:104370005C81CA01B9010E949C352D853E854F851F
:1043800058890E94F338A70196010E949C350E942B
:1043900092396093B3037093B4038093B503909301
:1043A000B6031CC032E03093AA0318C01092BB03BE
:1043B0001092BC031092BD031092BE038091B7030C
:1043C0009091B803A091B903B091BA038093B3035D
:1043D0009093B403A093B503B093B6031860109301
:1043E0000E0280913D03482F50E05A8B498B87E0A5
:1043F000849FF001859FF00D1124ED5EFC4F8091AC
:1044000098038483A091EF06B091F006BCAFABAFE8
:104410005E96BC91BAA3EBADFCADF78DFBA3ABAD43
:10442000BCAD9096BC91BCA3EBADFCADF1A1FDA3DE
:104430002091A6033091A7034091A8035091A903AE
:104440006AA17BA18B2F9F2F0E949B356EA77FA710
:1044500088AB99AB20E030E0A9010E94913687FF3C
:1044600004C01EA61FA618AA19AA2091B3032E8B5A
:104470003091B4033F8B4091B503488F5091B60300
:10448000598F8091BB038A8F9091BC039B8FA09121
:10449000BD03AC8FB091BE03BD8FE091AF03E98344
:1044A000F091B003FD832091B10329873091B203CD
:1044B0003D874091BF034EA35091C0035FA38091FD
:1044C000C10388A79091C20399A7A091AA03AD8BBD
:1044D000B091AB03BAA7E091AC03EBA7F091AD03A9
:1044E000FCA72091AE032DA73091B7033BAB4091C1
:1044F000B8034CAB5091B9035DAB8091BA038EAB5E
:104500002EA13FA148A5592F6A8D7B8D8C8D9D8D45
:104510000E949136811103C092E09AAB02C0A1E0E3
:10452000AAAB3AA02BA01CA10DA18EE3C82E83EC50
:10453000D82E8EE2E82E89E3F82E412C512C320140
:10454000CE8EDF8EE8A2F9A23D89313009F4F2C0A7
:10455000ABADBCAD313008F47BC0333009F020C1C5
:104560005A962D913D914D915C915D97C701B60191
:104570000E94F3384B015C012E893F89488D598D8B
:1045800069817D8189859D850E949B359B01AC0158
:10459000C501B4010E94B33887FD31C02A8D3B8D1F
:1045A0004C8D5D8D6AA17BA18CA19DA10E949B3544
:1045B0009B01AC010E949C356B017C0129813D81EE
:1045C00049855D856E897F89888D998D0E949C358E
:1045D0009B01AC01C701B6010E949B366B017C01B7
:1045E000BE89B983EF89ED83F88DF987298D2D87F1
:1045F0003A8C2B8C1C8D0D8D31E03D8B51C120E010
:1046000030E040E05FE3C501B4010E94F3389B0154
:10461000AC0169817D8189859D850E949B35A701BB
:1046200096010E94F3389B01AC01632D722D812FFE
:10463000902F0E949B35362E272E182F092FA5016B
:10464000940169817D8189859D850E949B356DC01E
:104650005A962D913D914D915C915D97C701B601A0
:104660000E94F3384B015C0120E030E040E05FE362
:104670000E94F33829813D8149855D850E949C35E2
:10468000A70196010E94F3389B01AC01632D722DA6
:10469000812F902F0E949B35362E272E182F092F01
:1046A000262F372F482F592F6A8D7B8D8C8D9D8D0E
:1046B0000E94B33818168CF52A8D3B8D4C8D5D8D7C
:1046C0006AA17BA18CA19DA10E949B359B01AC019D
:1046D0000E949C356B017C0129813D8149855D8566
:1046E0006E897F89888D998D0E949C359B01AC01D4
:1046F000C701B6010E949B366B017C01BAA9BD8B34
:10470000EE89E983FF89FD83288D2987398D3D87CF
:104710003A8C2B8C1C8D0D8DC3C0A5019401698131
:104720007D8189859D850E949C3569837D838987EC
:104730009D87B6C02E893F89488D598DC701B60126
:104740000E94F3389B01AC01632D722D812F902FB5
:104750000E949B355B014C019B01AC016EA17FA1C6
:1047600088A599A50E94B33818160CF095C02EA103
:104770003FA148A559A5632D722D812F902F0E942E
:104780009B352E893F89488D598D0E949B366B0140
:104790007C013EA02FA018A509A542E04D8B80C04A
:1047A0005A962D913D914D915C915D97C701B6014F
:1047B0000E94F3384B015C0129813D8149855D856B
:1047C0000E94913687FF39C020E030E040E05FE38F
:1047D000C501B4010E94F3389B01AC0169817D8160
:1047E00089859D850E949B35A70196010E94F3381B
:1047F0009B01AC01632D722D812F902F0E949B3560
:104800006FAB78AF89AF9AAF2AA53BA54CA55DA544
:104810000E94B33818168CF4A501940169817D813A
:1048200089859D850E949B3569837D8389879D87C6
:104830003FA828AC19AD0AAD33C02AA53BA54CA5AD
:104840005DA5632D722D812F902F0E949B359B01BA
:10485000AC010E949C356B017C0129813D81498519
:104860005D856BA97CA98DA99EA90E949C359B01A1
:10487000AC01C701B6010E949B366B017C01BBA94C
:10488000B983ECA9ED83FDA9F9872EA92D873AA458
:104890002BA41CA50DA504C03A2C2B2C182D092DDA
:1048A000A7019601C301B2010E949C352B013C0176
:1048B0002E8D3F8D48A159A10E94913687FF07C0D8
:1048C000A30192016E8D7F8D88A199A11CC02EA598
:1048D0003FA548A959A9632D722D812F902F0E94C1
:1048E000B338181684F52EE333EC4EE259E36E8D9F
:1048F0007F8D88A199A10E949C356E8F7F8F88A3A0
:1049000099A3A30192010E949B356B017C01232D89
:10491000322D412F502F6AA57BA58CA59DA50E9405
:10492000913687FD11CE89819D81A985BD858093B2
:10493000AF039093B003A093B103B093B2033D894A
:104940003093AA030FC089819D81A985BD8580937D
:10495000AF039093B003A093B103B093B2034D891A
:104960004093AA03E091ED06F091EE069189911132
:1049700004C080910E0283FF3FC0ABADBCAD519629
:104980008C915197807349F19E96CD90DD90ED907A
:10499000FC90D1979923D1F02091C3033091C403A7
:1049A0004091C5035091C6036091AF037091B0036D
:1049B0008091B1039091B2030E94F3389B01AC0146
:1049C000C701B6010E94F3386B017C01C701B60133
:1049D0000E9465028093C7030AC0109217021092CA
:1049E00018021092190210921A021092C7038091B5
:1049F0000E02877F80930E0247E029893A89429F01
:104A0000F001439FF00D1124ED5EFC4FFA87E9871A
:104A10008091C70386832091A2033091A303409124
:104A2000A4035091A503632D722D812F902F0E9416
:104A3000F33869837A838B839C830E947A366B0177
:104A40007C0160919E0370919F038091A0039091DF
:104A5000A1030E947A364B015C01A70196010E94D6
:104A60009B350E9414376D837E838F839887ED81F9
:104A7000FE81A985BA85ED93FC93EF2B41F48091DB
:104A80000E0281FF04C0816080930E020EC120914E
:104A90009A0330919B0340919C0350919D03C30165
:104AA000B2010E949C352B013C0129813A814B8146
:104AB0005C81C501B4010E949B359B01AC01C3011F
:104AC000B2010E949B364B015C0120EC31EE44E6C2
:104AD0005EE40E94F3380E947A360E941437603DEB
:104AE00037E073078105910560F4A7E049895A8989
:104AF000A49FF001A59FF00D1124ED5EFC4F1582DF
:104B000053C0603ABFE07B078105910560F447E040
:104B100029893A89429FF001439FF00D1124ED5EEF
:104B2000FC4F51E011C06034AFE17A078105910577
:104B300068F447E029893A89429FF001439FF00DCC
:104B40001124ED5EFC4F52E055830CC027E0A9898B
:104B5000BA892A9FF0012B9FF00D1124ED5EFC4FC6
:104B600033E03583A7E049895A89A49FF001A59FC6
:104B7000F00D1124ED5EFC4F2581022E04C09695A8
:104B80008795779567950A94D2F74D815E8102C02B
:104B9000440F551F2A95E2F7518340836115710533
:104BA00051E08507910568F427E0A989BA892A9F11
:104BB000F0012B9FF00D1124ED5EFC4F7383628397
:104BC00004C04FEF5FEF538342838091EC068093E4
:104BD0003D038F5F863019F08093EC0602C010927F
:104BE000EC06E091EF06F091F006832D922DA12FB7
:104BF000B02F868F978FA0A3B1A3C0929E03D092AF
:104C00009F03E092A003F092A10329813A814B8196
:104C10005C81C701B6010E949B35A50194010E94E9
:104C2000F33860939A0370939B0380939C03909353
:104C30009D032091AB033091AC034091AD035091A3
:104C4000AE03632D722D812F902F0E94913681111A
:104C5000A5C820E030E0A901632D722D812F902F8F
:104C60000E94B33890910E02181614F092FF04C0FF
:104C7000916090930E0219C01092F0061092EF0608
:104C80009091CA038091EB06891709F487C881E0E7
:104C9000890F803109F480E02091C803921302C08B
:104CA0008093C8038093CA0379C8EC960FB6F89432
:104CB000DEBF0FBECDBFDF91CF911F910F91FF904F
:104CC000EF90DF90CF90BF90AF909F908F907F90AC
:104CD0006F905F904F903F902F900895CF93DF9308
:104CE000C091EF06D091F0062097C9F0809199030A
:104CF0008160809399036091AF037091B0038091BC
:104D0000B1039091B2039B01AC010E94F3386A8B0E
:104D10007B8B8C8B9D8B1092F0061092EF06DF91AF
:104D2000CF9108952F923F924F925F926F927F9210
:104D30008F929F92AF92BF92CF92DF92EF92FF92AB
:104D40000F931F93CF93DF933090EB06311002C087
:104D5000D0E101C0D32DD150C091C803CD1709F4C3
:104D600016C1ED2EF12C22E3D29F800111240553B0
:104D70001C4FF801A688B788C08CD18C628D738DCA
:104D8000848D958D9B01AC010E949C35F801268D88
:104D9000378D40A151A10E94F3384B018C019B013A
:104DA000AC01B501C6010E94913687FD02C05401D5
:104DB000680182E38E9DF0018F9DF00D1124E55373
:104DC000FC4FC501D601828B938BA48BB58BD1117F
:104DD00001C0D0E1D150CD1307C08091CA03C813E0
:104DE00068C00E946E2665C022E32E9DC0012F9DE3
:104DF000900D11249C0125533C4F790192E3292EFB
:104E0000AD2EB12C2A9CC0012B9C900D1124FC01CD
:104E1000E553FC4F6F01D11101C0D0E1D150809119
:104E2000CA038D1302C00E946E262A9C80012B9C0F
:104E3000100D112405531C4FF80186889788A08C0B
:104E4000B18CA501940162897389848995890E9436
:104E50009136882359F1F801628D738D848D958D7B
:104E60009B01AC010E949C35F801268D378D40A135
:104E700051A10E94F338F701228933894489558969
:104E80000E949C352B013C019B01AC01C501B40182
:104E90000E94B338F80118162CF4428A538A648AA7
:104EA000758A04C0828A938AA48AB58A7601CD1352
:104EB000A7CFF2E3CF9F8001112405531C4FCF5F92
:104EC000C03109F4C0E0D091C80382E3282EC31595
:104ED00009F45BC0CC2ED12C2C9CC0012D9C900DD4
:104EE00011249C0125533C4F7901F80142885388D5
:104EF00064887588F90182889388A488B588A5019B
:104F00009401C301B2010E94913687FF24C0F801C9
:104F1000628D738D848D958D9B01AC010E949C35B3
:104F2000F801268D378D40A151A10E94F338A301CD
:104F300092010E949C352B013C019B01AC01C501F3
:104F4000B4010E94B338181634F4F701428A538A28
:104F5000648A758ADC2F2C9CF0012D9CF00D1124A5
:104F6000E553FC4F26893789408D518D62897389BD
:104F7000848995890E949136811101C0DC2FCF5F11
:104F8000C03109F4C0E08701A2CFD093C803DF91FC
:104F9000CF911F910F91FF90EF90DF90CF90BF9036
:104FA000AF909F908F907F906F905F904F903F90C9
:104FB0002F9008952F923F924F925F926F927F921F
:104FC0008F929F92AF92BF92CF92DF92EF92FF9219
:104FD0000F931F93CF93DF93CDB7DEB7C454D1099E
:104FE0000FB6F894DEBF0FBECDBF3B010091EB06BC
:104FF000202E312C22E3229DA001239D500D11244F
:10500000BA0165537C4F7AAF69AFFB0111922A95C3
:10501000E9F7F3012085FB01218BF30144815581E0
:1050200066817781E9ADFAAD46A757A760AB71AB52
:1050300021FF40C02CE0E1EFF1E0DE015996019044
:105040000D922A95E1F78BAB9CAB2BE132E03EABA6
:105050002DABBE01635F7F4F23967FAF6EAF23976B
:10506000CE01499621969FAF8EAF2197E2E30E9F26
:10507000C00111249C0125533C4F3EAF2DAF685E0B
:105080007F4F7CAF6BAF78AF6FAB10E082E3829D58
:105090009001839D300D1124C90185539C4FFC0163
:1050A0003C962596FFAFEEAF25972C01F0E14F0E11
:1050B000511C3CC02CE0E1EFF6E0BFCFEDADFEAD02
:1050C0002193319341935193FEAFEDAF2596EEAD11
:1050D000FFAD2597C080D180E280F380C216D30651
:1050E000E406F50610F469017A012596EEADFFADF0
:1050F0002597C082D182E282F3820E944537A501C2
:1051000094010E949B36EFA9F8AD6193719381934E
:105110009193F8AFEFAB20E030E0A9010E94913607
:1051200087FD42C01F5F133009F44CC0EBA9FCA9F6
:105130006191719181919191FCABEBABEDA9FEA9CD
:1051400081909190A190B190FEABEDABA50194013F
:105150000E94F3380E94C0382396EEADFFAD23972E
:1051600061937193819391932396FFAFEEAF239751
:105170002196EEADFFAD2197C190D190E190F190D5
:105180002196FFAFEEAF21976C197D098E099F091B
:105190009B01AC0197FF92CF22273327A901261B41
:1051A000370B480B590B8ACF112321F0113021F016
:1051B00080E803C080E201C080E4F2019081892B85
:1051C0008083B0CFCD28CE28CF2809F496C1CE0158
:1051D00085960E9479314B015C0122E3229DC0013A
:1051E000239D900D11249C0125533C4F7901F90119
:1051F000868E978EA0A2B1A2BE016B5D7F4F83E326
:1052000092E00E942331F701628F738F848F958F14
:10521000BE016B5D7F4F87E292E00E942331F70170
:1052200066A377A380A791A7118910FD12C0F3018F
:10523000208131814281538113FD06C0F70122A7ED
:1052400033A744A755A709C0C501B4010E94F3388C
:10525000F70162A773A784A795A78091CA030817CF
:1052600011F011FF0DC082E3829DF001839DF00DCE
:105270001124E553FC4F128A138A148A158A54C0EC
:105280002DEF36E03CAB2BAB8E010F5F1F4FBE0105
:105290006F5C7F4F7AAB69ABC12CD12C76010DAB23
:1052A0001FABEBA9FCA981909190A190B190FCABB0
:1052B000EBABEBADFCAD4190519061907190FCAFC8
:1052C000EBAFA3019201C501B4010E94F3389B0129
:1052D000AC01C701B6010E949B356B017C01A501A1
:1052E0009401C301B2010E949B35F801619371934F
:1052F000819391938F0129A93AA96BAD7CAD2617B3
:10530000370779F62FEE3FEF4FE75FE3C701B601AE
:105310000E94B33818166CF482E3829DF001839DDD
:10532000F00D1124E553FC4F12A213A214A215A2F2
:1053300071C02FEE3FEF4FE75FEBC701B6010E9450
:10534000913687FF11C082E3829DF001839DF00DAD
:105350001124E553FC4F89E996E7A6E9BEE782A34D
:1053600093A3A4A3B5A356C08DA99FA90E94793188
:105370006DA97FA983E392E00E9423314B015C0178
:10538000A701960160E070E080E89FE30E949B35F2
:1053900020E030E040E05FE30E94F3380E94923961
:1053A0006B017C01209150023091510240915202D8
:1053B00050915302C501B4010E94F338A701960130
:1053C0000E94F3384B015C01A701960160E070E098
:1053D00080E89FE30E949B359B01AC01C501B401AD
:1053E0000E949B366B017C0120E030E0A9010E9405
:1053F000913687FF03C0C12CD12C760182E3829DB8
:10540000F001839DF00D1124E553FC4FC2A2D3A2FD
:10541000E4A2F5A282E3829D8001839D100D1124F8
:1054200005531C4FF801818981FD69C089AD9AAD92
:105430000E94F41C6B017C018090090790900A0780
:10544000A0900B07B0900C07A50194010E94B338FF
:1054500018162CF4A5019401C501B40104C0A701DC
:105460009601C701B6010E94F338F801668B778B6D
:10547000808F918F82E3829D8001839D100D112486
:1054800005531C4FF80182A093A0A4A0B5A0A501CC
:10549000940166897789808D918D0E94B3381816A2
:1054A0002CF4F801868A978AA08EB18EC0920907E3
:1054B000D0920A07E0920B07F0920C078CE0FE01F5
:1054C000B596ADEFB6E001900D928A95E1F78CE0CC
:1054D000FE013D96A1EFB6E001900D928A95E1F7AD
:1054E0008091C9038093EB068F5F803109F480E0DF
:1054F0008093C9030E94922602C080E001C081E02F
:10550000CC5BDF4F0FB6F894DEBF0FBECDBFDF918F
:10551000CF911F910F91FF90EF90DF90CF90BF90B0
:10552000AF909F908F907F906F905F904F903F9043
:105530002F900895CF93DF930E94513280E3E8E9E2
:10554000F3E0DF011D928A95E9F7CFEED2E083E226
:10555000FE0111928A95E9F71092F0061092EF067B
:105560001092120310923D0381E08093EC0610929A
:10557000EE020E9420328091ED028F878BB1837EF4
:105580009091EC02892B8BB98BB18F719091ED02C8
:10559000892B8BB9DF91CF910895CF93DF93C1E130
:1055A000D7E08991882319F00E943D02FACFDF915C
:1055B000CF910895CF93DF9321E5829FC0011124FD
:1055C000EC01DD5F40E550E0BE0181E197E00E9423
:1055D0004B1E892B69F4109211070E94020240E5CC
:1055E00050E061E177E0CE010E94881D80E001C0BB
:1055F00081E0DF91CF9108959FB7F8942091100733
:10560000822B809310079FBF08959FB7F894209135
:105610000F07822B80930F079FBF08959FB7F894C1
:1056200080930E079FBF08952FB7F89490910D07B0
:105630008095892380930D072FBF08959FB7F89415
:1056400020910D07822B80930D079FBF0895AF9285
:10565000BF92CF92DF92EF92FF920F931F93CF935F
:10566000DF93EC010FE312E05C018CE0A80EB11CAB
:10567000C990D990E990F99020E030E0A901C701E4
:10568000B6010E94B33818168CF0F80121913191BF
:10569000419151918F01C701B6010E94913687FD5A
:1056A00005C0CA15DB0521F780E001C081E0DF916C
:1056B000CF911F910F91FF90EF90DF90CF90BF900F
:1056C000AF9008958F929F92AF92BF92CF92DF9248
:1056D000EF92FF920F931F93CF93DF93EB012BE198
:1056E000E22E22E0F22E8C016B018CE0C80ED11C60
:1056F0006991799189919991F70181909190A19007
:10570000B1907F010E944537A50194010E949B360C
:10571000F80161937193819391938F01CC15DD050D
:1057200039F7DF91CF911F910F91FF90EF90DF90AC
:10573000CF90BF90AF909F908F9008950E940202EB
:1057400010921602089596B1892F877049F0892F1B
:105750008095817091FF826092FD03C084600895FE
:1057600080E008951F920F920FB60F9211242F938D
:105770003F934F935F936F937F938F939F93AF93D9
:10578000BF93CF93EF93FF930E94A32BC82F88233F
:1057900089F080FD0E945F03C2FF05C080910D0764
:1057A000826080930D07C1FF05C080910D0788605E
:1057B00080930D07FF91EF91CF91BF91AF919F9192
:1057C0008F917F916F915F914F913F912F910F90AA
:1057D0000FBE0F901F9018951092F00190916002EB
:1057E00097FD03C090E29093F001882331F09091EF
:1057F000F00180E289278093F00108958F929F92B3
:10580000AF92BF92CF92DF92EF92FF920F931F93CE
:10581000CF93DF93CDB7DEB72D970FB6F894DEBFE9
:105820000FBECDBF6B017C01042F20E030E0A90149
:105830000E94913687FF07C08DE20E943D02F7FA71
:10584000F094F7F8F094102F123060F020E030E080
:1058500048EC52E4C701B6010E94F3386B017C01A9
:105860001250F2CF00FF0AC020E030E040E251E4E5
:10587000C701B6010E94F3386B017C0120E030E0E3
:1058800040E05FE3C701B6010E949C350E940D37DE
:1058900010E03AE0832E912CA12CB12C61157105FA
:1058A0008105910591F0EE24E394F12CEC0EFD1EA0
:1058B000E10EF11CA50194010E941C3A605DF70104
:1058C0006083B901CA011F5FE9CF80E3101748F474
:1058D000E1E0F0E0EC0FFD1FE10FF11D80831F5FA1
:1058E000F5CF101313C0FE01E10FF11D80E381839A
:1058F0001F5F0CC0101303C08EE20E943D02FE0128
:10590000E10FF11D80810E943D0211501111F2CF73
:105910002D960FB6F894DEBF0FBECDBFDF91CF91AD
:105920001F910F91FF90EF90DF90CF90BF90AF90BD
:105930009F908F9008952091600220FF08C02BE86F
:1059400032E441E25DE30E94F33841E001C040E00F
:105950000C94FE2B2091600220FF08C02BE832E45B
:1059600041E25DE30E94F33844E001C043E00C945F
:10597000FE2B0F931F93CF938C01C0E0F801619130
:105980007191819191918F010E94AA2CC23019F0DE
:105990008CE20E943D02CF5FC33081F7CF911F910F
:1059A0000F910895CF93DF93843630F06AE00E9420
:1059B000FC39C0E3C90F03C0C0E08A3030F06AE0B0
:1059C0000E94FC39D0E3D90F01C0D0E0805D0E9475
:1059D0003D02DD2319F08D2F0E943D02CC2329F0DA
:1059E0008C2FDF91CF910C943D02DF91CF910895E0
:1059F000CF93DF93FC018491EF012196882321F05E
:105A00000E943D02FE01F7CFDF91CF91089581E61C
:105A100093E00C94F82CCF93C82F8AE693E00E9471
:105A2000F82C8C2F0E94D22CCF910C94072D811131
:105A300004C081E793E00C94F82C0C940B2DCF93C9
:105A4000DF93C0E08C2F0E94DA2A81110EC01092E1
:105A500011078EE30E943D020E94CD2A8AE30E9434
:105A60003D0287E00E940B2D12C080911107882310
:105A700071F00E94C909D82F8EE30E943D020E9456
:105A8000CD2A8AE30E943D028D2F0E94172DCF5F01
:105A9000C230C1F6DF91CF910895CF92DF92EF929D
:105AA000FF92CF93DF93D82F6A017B01C22F84E24C
:105AB0000E943D028D2F0E94D22C8DE30E943D0258
:105AC0004C2FC701B6010E94FE2BDF91CF91FF90B2
:105AD000EF90DF90CF900C94072DCF93DF93D82FCA
:105AE000C62F84E20E943D028D2F0E94D22C8DE3AE
:105AF0000E943D028C2F0E94D22CDF91CF910C94FA
:105B0000072DEF92FF920F931F93CF93DF93609136
:105B10004B0270E080E00E946D2D60914E0270E0BB
:105B200081E00E946D2D60914C0270E082E00E9445
:105B30006D2D60914D0270E083E00E946D2D6091AB
:105B4000600262FB662760F970E084E00E946D2DC0
:105B50006091600266FB662760F970E085E00E9454
:105B60006D2D80916002082E000C990B692F661F25
:105B70006627661F70E086E00E946D2D60914F02DF
:105B800070E08AE00E946D2D4091500250915102C8
:105B9000609152027091530223E08BE00E944D2DE0
:105BA00040915402509155026091560270915702F3
:105BB00023E08CE00E944D2D60916002617070E0E6
:105BC0008DE00E946D2D6091600265FB662760F993
:105BD00070E084E10E946D2D6091600263FB662796
:105BE00060F970E085E10E946D2D60916002629520
:105BF000617070E086E10E946D2D6091610270E03D
:105C000087E10E946D2D4091620250916302609184
:105C100064027091650223E088E10E944D2D40915D
:105C2000660250916702609168027091690223E0F8
:105C300089E10E944D2D60916A0270916B028AE1A8
:105C40000E946D2D40916C0250916D0260916E0228
:105C500070916F0223E08BE10E944D2D409158021C
:105C60005091590260915A0270915B0220E08EE1DE
:105C70000E944D2D40915C0250915D0260915E0248
:105C800070915F0220E08FE10E944D2D60916002D3
:105C90006695617070E080E20E946D2DD4E6F12C73
:105CA0000BE112E083E0E82EED0ECD2F82E0F81636
:105CB00091F0E3E0FE16E9F0F1E0FF1631F0F801B3
:105CC00040815181628173811AC0F80144855585F4
:105CD0006685778514C020E030E041E655E4F801A0
:105CE000608D718D828D938D0E949B36AB01BC01BE
:105CF00006C0F80144A155A166A177A1705823E020
:105D00008C2F0E944D2D0C5F1F4FCF5FEC12CECF1A
:105D1000D65FF394DC3821F6DF91CF911F910F917C
:105D2000FF90EF9008958DE50E943D020C94072DA1
:105D3000CF93DF93CDB7DEB72C970FB6F894DEBFC5
:105D40000FBECDBF84E693E00E94F82C6DEF71E0AA
:105D5000CE0101960E94622BCE0101960E94B92CC1
:105D60008AE30E943D0280910F020E94D22C0E9481
:105D7000932E2C960FB6F894DEBF0FBECDBFDF91E9
:105D8000CF9108951F920F920FB60F9211242F9367
:105D90003F934F935F936F937F938F939F93AF93B3
:105DA000BF93EF93FF9380910A02813049F0809175
:105DB0000E07811105C00E945F0381E00E940E2B37
:105DC000FF91EF91BF91AF919F918F917F916F91D3
:105DD0005F914F913F912F910F900FBE0F901F90A9
:105DE000189593B196718091600286FD02C086E19C
:105DF0009827992349F091FB882780F992FD8260CA
:105E0000907119F08460089580E008952F923F9278
:105E10004F925F926F927F928F929F92AF92BF92BA
:105E2000CF92DF92EF92FF920F931F93CF93DF9366
:105E3000CDB7DEB7A1970FB6F894DEBF0FBECDBFCA
:105E400090910B029111C4C18F8FFE013D9689E0A4
:105E5000DF011D928A95E9F786E08D8BEBE1F2E098
:105E6000FA8FE98F5F019E012A5E3F4F490100E0F2
:105E700010E0C12CD12C76019F8D892F90E09E8F50
:105E80008D8F802F002321F0013021F090E103C09D
:105E900094E001C098E0D4019D934D01ED8DFE8DFD
:105EA00002C0F595E7958A95E2F7E0FF1BC020E078
:105EB00030E040EC5FEBD50194966D917D918D9132
:105EC0009C9197970E94F338362E472E582E692EB4
:105ED000A70196010E94913687FD04C0C32CD42CE3
:105EE000E52CF62C0F5F1F4FB4E0AB0EB11C033056
:105EF000110539F6209066023090670240906802E2
:105F00005090690284E0A82EBB24B39461EF71E045
:105F1000CE0101960E94622B80916102682E712C45
:105F2000FE01319621EF31E03C8F2B8F39A328A35E
:105F3000DE0156964D0180E090E000E010E0B701F0
:105F4000A60170582D8D3E8D082E02C035952795DF
:105F50000A94E2F720FF22C00F5FA8A1B9A11D9209
:105F60001D921D921C9213979301082E02C0359525
:105F700027950A94E2F720FF03C0BB2019F007C061
:105F8000BB2029F0C082D182E282F38204C0408328
:105F9000518362837383D4012C91122B0196BFEF3E
:105FA0008B1A9B0A349628A139A12C5F3F4F39A345
:105FB00028A38330910531F6602F70E080E090E0F7
:105FC0000E9443370E9492399B01AC01109310024A
:105FD000C201B1010E94F3386D877E878F87988B4D
:105FE000BE01635F7F4FCE0101960E94DA2734E045
:105FF00030930E020E94B01E0E94CF34BB20E9F005
:106000000E94F12EFE01769620E030E090E0619152
:10601000462F412359F0AC01022E02C055954795F9
:106020000A94E2F740FF02C0609516232F5F3F4FAE
:106030002330310561F7109310020E94B01E809149
:106040000D07847339F110910D0714FF03C086E02A
:106050000E940E2B15FF03C087E00E940E2BB1108B
:1060600007C00E94F12E9F8D892339F088E003C07C
:1060700012FF03C089E00E940E2B80910E07882337
:1060800029F00E945F030E94B61BA2C084E00E9418
:10609000142B04C0812F8C7109F0B0CF0E949A2A72
:1060A00000916A0210916B020115110549F0AFE9E8
:1060B000BFE01197F1F700C0000001501109F4CFC3
:1060C000B1E0BB26C9F020E030E040EA50E4609146
:1060D0006C0270916D0280916E0290916F020E942D
:1060E000F3386B017C012090620230906302409093
:1060F00064025090650210C0C0906C02D0906D0296
:10610000E0906E02F0906F0220906602309067027D
:106110004090680250906902AA94A110F7CEE090D6
:106120006102F12C80906C0290906D02A0906E0242
:10613000B0906F022401350177FA709477F870946B
:106140008D8D9E8D002E02C0959587950A94E2F75D
:1061500080FF2BC0C701002E02C0959587950A9439
:10616000E2F7E98DFA8D80FF0FC024A135A146A189
:1061700057A1C501B4010E949C35A98DBA8D2D91FE
:106180003D914D915C9106C02081318142815381C6
:10619000C301B2010E94F3380E94C038AB8DBC8DA0
:1061A0006D937D938D939C9313970F5F1F4FEB8D92
:1061B000FC8D3496FC8FEB8F298D3A8D2C5F3F4FF1
:1061C0003A8F298F0330110509F0BACF10920E02D1
:1061D000A1960FB6F894DEBF0FBECDBFDF91CF9171
:1061E0001F910F91FF90EF90DF90CF90BF90AF90F5
:1061F0009F908F907F906F905F904F903F902F90E7
:106200000895EBE6F0E08081897E8083E8E6F0E0A7
:1062100080818E7F8083089584B1897E84B985B121
:10622000866185B98091600283FF0BC080916B000D
:10623000866180936B008091680081608093680024
:1062400008950C9401316F927F928F929F92AF923A
:10625000BF92CF92DF92EF92FF920F931F93CF9353
:10626000DF93EB018C015B018CE0A80EB11C89E986
:10627000682E96E7792E26E9822E3EE7932EC99066
:10628000D990E990F99020E030E0A901C701B6016A
:106290000E9491368823B9F0A7019601F801608128
:1062A0007181828193810E949B366B017C01E8940D
:1062B000F7F89301A401C701B6010E94B33818167C
:1062C00014F0360147010C5F1F4FCA15DB05B9F604
:1062D000B301C401DF91CF911F910F91FF90EF9017
:1062E000DF90CF90BF90AF909F908F907F906F90F6
:1062F00008954F925F926F927F92AF92BF92CF922A
:10630000DF92EF92FF920F931F93CF93DF93EC01F5
:106310005C018CE0A80EB11C8E01C12CD12C760141
:10632000F80141905190619071908F0120E030E030
:10633000A901C301B2010E949136882371F0A30123
:106340009201C301B2010E94F3389B01AC01C70165
:10635000B6010E949C356B017C010A151B0501F7F3
:10636000C701B6010E9492396B017C019B01AC010F
:1063700060E070E080E89FE30E949B362B013C01C7
:10638000A3019201688179818A819B810E94F338FF
:106390006993799389939993AC16BD0689F7C701E0
:1063A000B601DF91CF911F910F91FF90EF90DF9099
:1063B000CF90BF90AF907F906F905F904F90089577
:1063C0001F93CF93DF93142F20E030E040EA51E495
:1063D0000E94F3380E947A360E941437EB0120970E
:1063E000D1F080910B02811116C0111103C00E94DF
:1063F000B61B06C00E94741780910C0281FD0BC071
:106400002FEF80E792E0215080409040E1F700C0FC
:1064100000002197E4CFDF91CF911F910895E1EF24
:10642000F1E0A1EFB6E041915191619171914D93ED
:106430005D936D937D9381E0ED3FF807A1F708959B
:1064400080914C02682F20914D02422F982F91701D
:1064500080FD94E0822F817020FD80E261FD9860D4
:1064600041FD806462FD906142FD80689093EC0282
:106470008093ED0208951F920F920FB60F92112490
:106480008F939F938BB19091EC029C71837E892BAB
:106490008BB915BC9F918F910F900FBE0F901F90DD
:1064A000189580916F008D7F80936F00809181009F
:1064B000887F8160809381001092EE0280914E026D
:1064C00090910A028F3F39F420910E07211103C0E9
:1064D000903881F402C0943069F090E0009741F068
:1064E000EFE9FFE03197F1F700C000000197F6CF28
:1064F00081E001C080E09091600292FF02C091E0D3
:106500008927882311F0289A0895289808951F92C2
:106510000F920FB60F9211242F933F934F935F93D7
:106520006F937F938F939F93AF93BF93EF93FF935B
:106530008091EE02811122C28BB19091FE02907E79
:106540008F71892B8BB98BB1837E9091FD02892B42
:106550008BB98091FC0286BD82E085BD81E080938D
:10656000EE0278948091100390911103892B09F029
:10657000BFC08091120390913D03981709F4A4C005
:10658000E09112032E2F30E087E0E89FF001112404
:10659000ED5EFC4FF0931103E09310038281938131
:1065A00090938900809388008081918190930C035F
:1065B00080930B03E48180910D038E1761F1E093CA
:1065C0000D0382E1E89FF0011124E25CFC4FF0939F
:1065D0000F03E0930E0384859585A685B785B69550
:1065E000A795979587958093F7029093F802A093CB
:1065F000F902B093FA028093F3029093F402A0930D
:10660000F502B093F6028093EF029093F002A0930C
:10661000F102B093F202A0910E03B0910F035096D5
:106620009C9150978091ED0289278093FE0287E02C
:10663000829FF001839FF00D1124ED5EFC4F2581B8
:106640004D915D916D917C911397022E04C07695CA
:106650006795579547950A94D2F74093FF02509358
:106660000003609301037093020314964D915D91B2
:106670006D917C911797022E04C07695679557957A
:1066800047950A94D2F74093030350930403609311
:1066900005037093060318968D919D910D90BC9102
:1066A000A02D04C0B695A795979587952A95D2F702
:1066B0008093070390930803A0930903B0930A0300
:1066C00086810E94020314C00E945132E0910E03A1
:1066D000F0910F038189882339F01092B3008091E3
:1066E000B0008F778093B00084E00E941E2B46C1DB
:1066F000809109028130B1F486B180729091F001ED
:10670000891781F0109209028CE0E1EFF1E0ADEF22
:10671000B1E001900D928A95E1F780910D078064B8
:1067200080930D071092FD024091EF025091F0020C
:106730006091F1027091F2028091FF02909100034A
:10674000A0910103B0910203840F951FA61FB71FEC
:106750008093EF029093F002A093F102B093F202C3
:10676000E0910E03F0910F0344855585668577858A
:10677000481759076A077B0768F524E02093FD0254
:106780004485558566857785841B950BA60BB70BCD
:106790008093EF029093F002A093F102B093F20283
:1067A00020898091F1019091F201A091F301B091C3
:1067B000F40125FF04C00197A109B10903C00196A6
:1067C000A11DB11D8093F1019093F201A093F301FB
:1067D000B093F4014091F3025091F4026091F502FC
:1067E0007091F6028091030390910403A091050338
:1067F000B0910603840F951FA61FB71F8093F30265
:106800009093F402A093F502B093F6024485558567
:1068100066857785481759076A077B0778F52091C1
:10682000FD0228602093FD024485558566857785A5
:10683000841B950BA60BB70B8093F3029093F40285
:10684000A093F502B093F60220898091F501909112
:10685000F601A091F701B091F80126FF04C001975D
:10686000A109B10903C00196A11DB11D8093F501D5
:106870009093F601A093F701B093F8014091F702CD
:106880005091F8026091F9027091FA028091070329
:1068900090910803A0910903B0910A03840F951FFA
:1068A000A61FB71F8093F7029093F802A093F902F6
:1068B000B093FA0244855585668577854817590750
:1068C0006A077B0778F52091FD0220612093FD0285
:1068D0004485558566857785841B950BA60BB70B7C
:1068E0008093F7029093F802A093F902B093FA0212
:1068F00020898091F9019091FA01A091FB01B0915A
:10690000FC0127FF04C00197A109B10903C001964A
:10691000A11DB11D8093F9019093FA01A093FB0191
:10692000B093FC0180910A02843039F49091FD0209
:106930008091100289238093FD0280910B03909136
:106940000C03019790930C0380930B03892B69F43C
:106950001092110310921003809112038F5F8093A5
:106960001203863011F4109212039091FD0280916F
:10697000EC0289278093FD021092EE02FF91EF91C5
:10698000BF91AF919F918F917F916F915F914F9147
:106990003F912F910F900FBE0F901F9018958091EF
:1069A000600282FF02C0289A01C028988091EC0200
:1069B0008093FD0280914B02880F845081958093D3
:1069C000FC0280916F00826080936F0008958F9227
:1069D0009F92AF92BF92CF92DF92EF92FF920F936E
:1069E0001F93CF93DF937C016B01DC01CC91D0E04E
:1069F000FE01EF5EF84F80818D3229F4EF0122967F
:106A0000818101E009C08B3219F0CE5ED84F03C0FE
:106A1000EF012296818100E0912CF0E010E020E06F
:106A200030E0A9015E01E0EDE80FEA30D0F4FF5F4D
:106A3000F93098F491101150A5E0B0E00E94443A6A
:106A4000DC01CB01880F991FAA1FBB1F9C01AD0160
:106A50002E0F311D411D511D0AC0911008C01F5F2E
:106A600006C0EE3F41F4911006C0992493942196FC
:106A7000D5018C91D7CFFF2309F44FC0CA01B901CA
:106A80000E9443374B015C0120E030E0A9010E94E5
:106A90009136882349F11F3F64F42AE037ED43E241
:106AA0005CE3C501B4010E94F3384B015C011E5F39
:106AB000F2CF1F3F59F42DEC3CEC4CEC5DE3C501EB
:106AC000B4010E94F3384B015C010EC0112361F048
:106AD00020E030E040E251E4C501B4010E94F33807
:106AE0004B015C011150F2CF002351F0B7FAB09482
:106AF000B7F8B094F60180829182A282B38206C078
:106B0000D6018D929D92AD92BC921397C151D74000
:106B1000C150F701C08381E001C080E0DF91CF91D7
:106B20001F910F91FF90EF90DF90CF90BF90AF90AB
:106B30009F908F9008955058BB27AA270E94B33585
:106B40000C944D380E94143838F00E941B3820F005
:106B500039F49F3F19F426F40C94EA370EF4E095CB
:106B6000E7FB0C94BB37E92F0E94723858F3BA1731
:106B7000620773078407950720F079F4A6F50C9453
:106B8000AC380EF4E0950B2EBA2FA02D0B01B901F5
:106B900090010C01CA01A0011124FF27591B99F093
:106BA000593F50F4503E68F11A16F040A22F232F9F
:106BB000342F4427585FF3CF469537952795A795EF
:106BC000F0405395C9F77EF41F16BA0B620B730B96
:106BD000840BBAF09150A1F0FF0FBB1F661F771F07
:106BE000881FC2F70EC0BA0F621F731F841F48F4BC
:106BF000879577956795B795F7959E3F08F0B0CF45
:106C00009395880F08F09927EE0F9795879508952B
:106C10000E94143860F080E891E009F49EEF0E9431
:106C20001B3828F040E851E071F45EEF0CC00C9482
:106C3000EA370C94AC38E92FE0780E94723840F3C0
:106C4000092E052AB1F3261737074807590738F0E8
:106C50000E2E07F8E02569F0E025E0640AC0EF6336
:106C600007F8009407FADB01B9019D01DC01CA01B4
:106C7000AD01EF930E94B2360E944D380E944B3610
:106C80005F91552339F02BED3FE049E450FD49EC8D
:106C90000C949C350895DF93DD27B92FBF7740E82A
:106CA0005FE31616170648075B0718F4D92F0E94F2
:106CB000B8389F938F937F936F930E94D239EEE001
:106CC000F1E00E94ED370E944D382F913F914F9196
:106CD0005F910E940639DD2351F09058A2EA2AED17
:106CE0003FE049EC5FE3D0785D270E94B335DF9148
:106CF0000C944D380E94943890F09F3748F49111CD
:106D000016F40C94AD3860E070E080E89FE30895DD
:106D100026F01B16611D711D811D0C94C1370C944A
:106D2000DC370E94973708F481E008950E942438E8
:106D3000E3950C945E380E94AF360C944D380E9457
:106D40001B3858F00E94143840F029F45F3F29F0B6
:106D50000C94BB3751110C94AD380C94EA370E9457
:106D6000723868F39923B1F3552391F3951B550BB2
:106D7000BB27AA2762177307840738F09F5F5F4F0E
:106D8000220F331F441FAA1FA9F335D00E2E3AF04D
:106D9000E0E832D091505040E695001CCAF72BD065
:106DA000FE2F29D0660F771F881FBB1F26173707B6
:106DB0004807AB07B0E809F0BB0B802DBF01FF27E8
:106DC00093585F4F3AF09E3F510578F00C94BB37D3
:106DD0000C94AD385F3FE4F3983ED4F386957795F5
:106DE0006795B795F7959F5FC9F7880F911D9695A1
:106DF000879597F90895E1E0660F771F881FBB1FFD
:106E0000621773078407BA0720F0621B730B840BA9
:106E1000BA0BEE1F88F7E09508950E941437689426
:106E2000B1110C94AD3808950E947A3888F09F57BC
:106E300098F0B92F9927B751B0F0E1F0660F771F9E
:106E4000881F991F1AF0BA95C9F714C0B13091F094
:106E50000E94AC38B1E008950C94AC38672F782FBD
:106E60008827B85F39F0B93FCCF386957795679559
:106E7000B395D9F73EF490958095709561957F4FC5
:106E80008F4F9F4F0895E89409C097FB3EF490956B
:106E90008095709561957F4F8F4F9F4F9923A9F0F3
:106EA000F92F96E9BB279395F69587957795679582
:106EB000B795F111F8CFFAF4BB0F11F460FF1BC0C6
:106EC0006F5F7F4F8F4F9F4F16C0882311F096E959
:106ED00011C0772321F09EE8872F762F05C0662307
:106EE00071F096E8862F70E060E02AF09A95660FC0
:106EF000771F881FDAF7880F9695879597F9089579
:106F00000E94943890F09F3748F4911116F00C9439
:106F1000AD3860E070E080E89FEB089526F41B1622
:106F2000611D711D811D0C94C1370C94DC37990FC4
:106F30000008550FAA0BE0E8FEEF16161706E80743
:106F4000F907C0F012161306E407F50798F0621B64
:106F5000730B840B950B39F40A2661F0232B242B39
:106F6000252B21F408950A2609F4A140A6958FEF58
:106F7000811D811D089597F99F6780E870E060E0AA
:106F80000895882371F4772321F09850872B762F6A
:106F900007C0662311F499270DC09051862B70E02D
:106FA00060E02AF09A95660F771F881FDAF7880F3E
:106FB0009695879597F908959F3F31F0915020F469
:106FC000879577956795B795880F911D96958795C5
:106FD00097F908959FEF80EC0895DF93CF931F9367
:106FE0000F93FF92EF92DF927B018C01689406C0B1
:106FF000DA2EEF010E940639FE01E894A591259151
:10700000359145915591A6F3EF010E94B335FE01EC
:107010009701A801DA9469F7DF90EF90FF900F9144
:107020001F91CF91DF91089500240A941616170638
:1070300018060906089500240A9412161306140669
:10704000050608950C94EA370E947A38D8F3E8943C
:10705000E0E0BB279F57F0F02AED3FE049EC06C087
:10706000EE0FBB0F661F771F881F28F0B23A62072A
:107070007307840728F0B25A620B730B840BE395F5
:107080009A9572F7803830F49A95BB0F661F771F78
:10709000881FD2F790480C94DE37092E0394000C19
:1070A00011F4882352F0BB0F40F4BF2B11F460FFA2
:1070B00004C06F5F7F4F8F4F9F4F0895EF93E0FFA6
:1070C00007C0A2EA2AED3FE049EC5FEB0E94B3352E
:1070D0000E944D380F90039401FC9058EBE3F1E0CF
:1070E0000C94E83957FD9058440F551F59F05F3FF5
:1070F00071F04795880F97FB991F61F09F3F79F0DA
:1071000087950895121613061406551FF2CF46955B
:10711000F1DF08C0161617061806991FF1CF8695DD
:1071200071056105089408950E947A38A0F0BEE7C1
:10713000B91788F4BB279F3860F41616B11D672F66
:10714000782F8827985FF7CF869577956795B11D3B
:1071500093959639C8F30895E894BB276627772757
:10716000CB0197F908950E94973708F48FEF08959F
:107170009B01AC0160E070E080E89FE30C949B36DB
:107180000E947A3858F19E5760F19851A0F0E9F0CA
:10719000983020F5092E9927660F771F881F991FB1
:1071A0000A94D1F712C0062E672F782F8827985F90
:1071B00011F4000C07C0993FB4F386957795679555
:1071C0009395D9F7611D711D811D3EF490958095B1
:1071D000709561957F4F8F4F9F4F089568940C94E1
:1071E000AD380C94AC380E9406390C944D380E948E
:1071F000143838F00E941B3820F0952311F00C94BD
:10720000BB370C94EA3711240C94AD380E947238C5
:1072100070F3959FC1F3950F50E0551F629FF001E9
:10722000729FBB27F00DB11D639FAA27F00DB11D02
:10723000AA1F649F6627B00DA11D661F829F22278B
:10724000B00DA11D621F739FB00DA11D621F839F12
:10725000A00D611D221F749F3327A00D611D231FE8
:10726000849F600D211D822F762F6A2F11249F5736
:1072700050409AF0F1F088234AF0EE0FFF1FBB1F39
:10728000661F771F881F91505040A9F79E3F5105F8
:1072900080F00C94BB370C94AD385F3FE4F3983E1C
:1072A000D4F3869577956795B795F795E7959F5FA2
:1072B000C1F7FE2B880F911D9695879597F9089534
:1072C0000E947A38E8F09E37E8F09639B8F49E3894
:1072D00048F4672F782F8827985FF9CF86957795A0
:1072E000679593959539D0F3B62FB1706B0F711DDB
:1072F000811D20F487957795679593950C94C137F8
:107300000C94DC370C94AD389F930E9424380F9076
:1073100007FCEE5F0C945E3819F416F40C94EA370F
:107320000C94DC370E947A38B8F39923C9F3B6F38A
:107330009F57550B87FF0E94E1390024A0E640EAE1
:10734000900180585695979528F4805C660F771FBA
:10735000881F20F026173707480730F4621B730B8D
:10736000840B202931294A2BA695179407942025B0
:1073700031254A2758F7660F771F881F20F02617F8
:107380003707480730F4620B730B840B200D311D57
:10739000411DA09581F7B901842F9158880F9695CA
:1073A000879508959B01AC010C94F3380E949438A2
:1073B00030F09F3710F40C94AD380C94C1370C9416
:1073C000DC3791505040660F771F881FD2F7089521
:1073D0009F938F937F936F93FF93EF939B01AC01E8
:1073E0000E94F338EF91FF910E94ED372F913F916A
:1073F0004F915F910C94F338991B79E004C0991F69
:10740000961708F0961B881F7A95C9F780950895FE
:10741000AA1BBB1B51E107C0AA1FBB1FA617B707BA
:1074200010F0A61BB70B881F991F5A95A9F78095D6
:107430009095BC01CD010895A1E21A2EAA1BBB1B99
:10744000FD010DC0AA1FBB1FEE1FFF1FA217B30730
:10745000E407F50720F0A21BB30BE40BF50B661F46
:10746000771F881F991F1A9469F76095709580950A
:1074700090959B01AC01BD01CF010895EE0FFF1F58
:107480000590F491E02D09940E944F3AA59F900D2C
:10749000B49F900DA49F800D911D11240895A29F6B
:1074A000B001B39FC001A39F700D811D1124911DD8
:1074B000B29F700D811D1124911D0895FB01DC0107
:1074C00004C08D910190801921F441505040C8F7BB
:0A74D000881B990B0895F894FFCF74
:00000001FF
